:020000040800F2
:10000000201600202D020008434A0008FD39000890
:10001000414A0008D5140008C56E00080000000021
:1000200000000000000000000000000085670008DC
:10003000A518000800000000C9640008A9670008AE
:10004000470200084702000847020008470200086C
:10005000470200084702000847020008470200085C
:10006000470200084702000847020008470200084C
:10007000470200084702000847020008470200083C
:100080005915000847020008470200084702000807
:10009000470200084702000847020008470200081C
:1000A00047020008096800084702000847020008E4
:1000B0004702000847020008470200084D3A0008BE
:1000C000413A0008470200084702000847020008BA
:1000D000E5650008516E0008856E0008A56E0008F1
:1000E00047020008470200084702000847020008CC
:1000F00047020008470200084702000847020008BC
:1001000047020008470200084702000847020008AB
:10011000470200084702000847020008470200089B
:10012000470200084702000847020008470200088B
:1001300000F002F800F06AF80AA090E8000C82448F
:100140008344AAF10107DA4501D100F05FF8AFF26C
:10015000090EBAE80F0013F0010F18BFFB1A43F0A5
:10016000010318474C9900006C9900000A444FF0B5
:10017000000C10F8013B13F0070408BF10F8014B06
:100180001D1108BF10F8015B641E05D010F8016B4B
:10019000641E01F8016BF9D113F0080F1EBF10F8AF
:1001A000014BAD1C0C1B09D16D1E58BF01F801CBD2
:1001B000FAD505E014F8016B01F8016B6D1EF9D555
:1001C0009142D6D37047000000230024002500266A
:1001D000103A28BF78C1FBD8520728BF30C148BFAA
:1001E0000B607047662908F00684642900F0668079
:1001F000002070471FB500F0D5FB0400002000214F
:1002000007F0FAFEE0601FBD10B510BD00F0CAFC9B
:100210001146FFF7EFFF07F0EBFA00F0E8FC03B43C
:10022000FFF7F2FF03BC00F02BFD000009488047F8
:1002300009480047FEE7FEE7FEE7FEE7FEE7FEE7C8
:10024000FEE7FEE7FEE7FEE704480549054A064BE0
:1002500070470000056800083101000820100020E8
:10026000201600202012002020120020B2F12003CE
:100270000AD5C2F1200320FA02F001FA03F321FAB1
:1002800002F140EA0300704721FA03F04FF0000149
:10029000704700000FB41CB5074B06AA7B446946A3
:1002A0000090059800F065FB0020694600F074FBA3
:1002B0001CBC5DF814FB0000F90600002DE9F041BC
:1002C0000646002410687529314616A510D0AFF3F4
:1002D0000080002802DA404213A507E031688A074F
:1002E00001D512A502E0490704D511A5012401E0BA
:1002F000AFF3008000210A2206F1240709E0B0FBD9
:10030000F2FCB0FBF2F302FB1C00303078541846CC
:10031000491C0028F3D123462A463046BDE8F04167
:1003200000F0B9B8000000002D0000002B00000014
:10033000200000002DE9F0474FF0000A89460446EE
:10034000C0F820A02046E1688847002876D02528FC
:1003500006D0D4E901219047206A401C2062F1E7D1
:10036000E168204600258847C4F81CA006460027FF
:10037000C4F818A02A2E09D0304606F08BFE38B3F8
:1003800004EB8708303EC8F8186019E059F8041BE0
:10039000204604EB87029161E1688847012F0646F9
:1003A00018D1E069002820DA25F020051DE0D8F8F2
:1003B000180000EB800006EB40003038C8F8180049
:1003C0002046E1688847064606F064FE0028EED124
:1003D000012F0AD02E2E08D12046E16888477F1CC5
:1003E0000646022F45F02005C4DBA069002803DA89
:1003F000404245F00105A061E80701D025F0100555
:10040000B6B1A6F14100192802D8203645F400659E
:100410004A463146204625604D46FFF7E3FE58B177
:10042000012806D0ED1D25F0070000F1080989E735
:1004300004E005F1040985E730468AE7206ABDE853
:10044000F0874FF0000200B51346944696462039D7
:1004500022BFA0E80C50A0E80C50B1F12001BFF47D
:10046000F7AF090728BFA0E80C5048BF0CC05DF8E3
:1004700004EB890028BF40F8042B08BF704748BF31
:1004800020F8022B11F0804F18BF00F8012B7047A5
:100490007047704770472DE9F0470D4699469246E0
:1004A000044600F124080168880604D5E06921F0BB
:1004B0001001216000E00120A84201DD471B00E09F
:1004C0000027A1697A1902EB0900081AA0612078B7
:1004D000C00602D42046AFF30080002608E0D4E92D
:1004E00001211AF806009047206A401C761C206201
:1004F0004E45F4DB2078C0060AD52046AFF30080D5
:1005000006E0D4E9012130209047206A401C206297
:10051000381EA7F10107F4DC07E0D4E9012118F83F
:1005200005009047206A401C2062281EA5F10105A5
:10053000F3DC2046AFF300802078000602D50220CD
:10054000BDE8F0870120FBE770472DE9FF4F0C461F
:100550001E464FF0FF378BB0D2E90001DDF8608016
:100560000A908A46C1F30A5505B93D46002108465E
:100570004FF00000BAF1000F00F4400005DA00EB84
:1005800080004FF4400101EA50004FEA9059B9F160
:10059000010F00DDB9460A9850EA4A000ED044F631
:1005A0001050A5F2FF3545432F14B8F1000F1ED0AF
:1005B0007542291E1EDDC9F100021CE0B8F1010FD1
:1005C0004FF0000001D0302103E0F24305E0215458
:1005D000401CB042FBDB30460022002121540B9925
:1005E000C1F80880C1E900200FB0BDE8F08FBD1B45
:1005F0006D1CDEE74A4600DA694206A800F05CFAA4
:1006000006AB93E8070003AB83E8070050460A995E
:1006100000F03DFB8DE80700A0F500501F3800906A
:100620000398002D0ADD42F21F014A4608440023C8
:1006300003A90390684600F0A6FD09E0A0F500506C
:100640004A461F38002303A90390684600F0B0FD16
:100650008DE807000004000C03D04FF0FF30410884
:1006600000E01046B8F1000F03D0002200921546BA
:100670001EE0751E05D400F099F9303262556D1EEA
:10068000F9D5B3460122084302D000227F1C04E0C2
:100690002078302801D100227F1E002A099784D0BB
:1006A0001DE0112D07DA00F081F9303262556D1C22
:1006B00050EA0102F5D1084302D00098C8B10EE01B
:1006C0000021681E05E0235C625C63542254401ED6
:1006D000491C8142F7DBAB46A81B401E0990002055
:1006E00004F80B000B98099AC0F80880C0E9002BA9
:1006F0007AE711264FF0000857E72DE9F04F8846BA
:100700000446D21D22F0070191B0D1E90001CDE9E4
:100710000A0106F09BFC02460B98C00F01D02D2069
:1007200007E02068810701D52B2002E0202101EAA3
:10073000C000032A099001D0072A05DB0346414681
:10074000204600F079F90BE12078800601D5E069B8
:1007500000E00620B8F1650F814606D0B8F1660FBB
:1007600018D0B8F1670F70D131E00020B9F1110F46
:10077000009001DB112301E009F101030AAA01A99C
:100780000CA8FFF7E2FEDDE90C70002609F1010577
:10079000834647E001204B4600904FF000470AAAED
:1007A00001A90CA8FFF7D1FEDDE90DB00C995D465B
:1007B000002610B909F101000D18B9EB050003D4AA
:1007C000C0F1FF3609F10105A5EB09002BE0B9F1F5
:1007D000010F01DA4FF001090020B9F1110F00906B
:1007E000484601DD112300E003460AAA01A90CA82E
:1007F000FFF7ABFEDDE90C704D46002683462078FE
:1008000000070AD4AB4500DA5D4601A8012D04DDDE
:10081000411911F8011C302907D04F4502DA17F1B0
:10082000040F04DA012082460FE06D1EEEE7002F70
:1008300002DCED1B3E4403E0781CA84200DD7D1C79
:10084000B81B00F1010A4FF000472078000703D4DD
:10085000AA4501DB4FF0FF3A0021B7F1004F0DF13F
:1008600043088DF8431024D002202B23002F01DAF7
:100870007F422D230A21021EA0F1010000DC5FB19E
:1008800097FBF1FC97FBF1F201FB1C7C17460CF186
:10089000300C08F801CDEEE7A8F1010003702188C3
:1008A000090501D5452100E06521A0F1010800F806
:1008B000011C09980FA9A1EB0807FF1D00B1012039
:1008C000411901EBEA70A1693844081A401EA06181
:1008D0002078C00602D42046AFF30080099828B1E2
:1008E000D4E901219047206A401C20622078C0068C
:1008F00022D52046AFF300801EE0002E04DBB34576
:1009000002DD01A8805D00E03020D4E9012190479C
:10091000206A401C2062761CAAF101005FEA000AEE
:100920000AD100F03FF8C0680168405CD4E90121B9
:100930009047206A401C2062281EA5F10105DCDCDE
:1009400007E0D4E9012118F8010B9047206A401C08
:100950002062381EA7F10107F3DC2046AFF30080C8
:10096000032011B041E6000001694A1C02610878C9
:10097000704700B58FB0CDE90131002105910549DF
:100980007944CDE9031011466846FFF7D3FC0FB058
:1009900000BD0000E5FFFFFF0A6802F8010B0A60D6
:1009A0007047000000487047E00F002030B5B0F1FC
:1009B0000A024FEA900E71F100034EEA817EB0EB1D
:1009C0000E0061EB91014FEA101E4EEA017E10EB22
:1009D0000E0041EB11114FEA102E4EEA016E10EBA2
:1009E0000E0041EB11214FEA104E4EEA014E10EB82
:1009F0000E0041EB1141401841F100014FEAD000D7
:100A000040EA41704FEAD10110EB80054FEA8104C2
:100A100044EA907444EB01046D1944EB0404521B46
:100A2000A3414FF0000348BF0A3200D530BD401C3F
:100A300041F1000130BD00002DE9F0411F460446A0
:100A400003260168072A01F4006004DB08B116A53B
:100A500005E016A503E008B115A500E015A521F0F5
:100A600010002060A069C01EA0610FB1401EA061EF
:100A70002046AFF300804FB1D4E9012138469047BA
:100A8000206A401C2062C01C206206E0206AFAE74F
:100A9000D4E9012115F8010B9047761EF8D22046C3
:100AA000AFF30080BDE8F0814E414E006E616E00F4
:100AB000494E4600696E66002DE9F04781461646AC
:100AC0008AB0354878440DC88DE80D003248784426
:100AD000801C03AC0DC884E80D0041F69B3008442F
:100AE000372190FBF1F290FBF1F5A5F1800501FBB8
:100AF00012041B3C02D56442012000E00020DFF814
:100B000098A080460027FA44AAF1BE0A0EE0E0074A
:100B10000AD03246684607EB470101230AEB810100
:100B200000F046FB8DE8070064107F1C002CEED11E
:100B3000194F7F44AE3F19E0E80715D007EB0410CA
:100B40000DF1180A90E80E008AE80E00C068F04225
:100B500001D1981908903246012306A903A800F094
:100B600027FB03AB83E807006D10641C002DE3D165
:100B70004FF0010332466946B8F1000F03A802D0D6
:100B800000F001FB01E000F013FBC9E90001C9F826
:100B900008200AB0BDE8F087D08F000000487047F9
:100BA000C00F00207546FFF7F9FFAE460500694605
:100BB000534620F00700854618B020B5FFF744FBE8
:100BC000BDE820404FF000064FF000074FF000084E
:100BD0004FF0000B21F00701AC46ACE8C009ACE8CF
:100BE000C009ACE8C009ACE8C0098D46704710B533
:100BF0000446AFF300802046BDE81040FFF70FBB6E
:100C00004FF0013C50F8042B51F8043B9A4221D19B
:100C1000A2EB0C03934313EACC1317D150F8042B27
:100C200051F8043B9A4215D1A2EB0C03934313EA0B
:100C3000CC130BD150F8042B51F8043B9A4209D144
:100C4000A2EB0C03934313EACC13DBD04FF000006C
:100C5000704700BFD01A01BAB1FA81F101F0180152
:100C600022FA01F0CB40C1F12001DBB2C0B2C01AC0
:100C70002CFA01F3D11A914311EAC311E6D170475E
:100C800001491820ABBEFEE72600020070475FEA6C
:100C9000400C08BF91F0000F4FEA8C234FEAC122AD
:100CA00043EA51514FEA1C5018BF00F5F0404FEA9B
:100CB000300018BF41F000415FEA6C5C00F0298011
:100CC000BCF1FF3F08BF40F080407047130C06BFE7
:100CD00012044FF0100C4FF0000C130E04BF120260
:100CE0000CF1080C130F04BF12010CF1040C930F4C
:100CF00004BF92000CF1020CD30F04BF52000CF1A0
:100D0000010C11464FF00002A0F11F00A0EB0C00F7
:100D1000704711F0004F08BF704731F000413FF4B9
:100D2000D5AF0B0C06BF09044FF0100C4FF0000CB0
:100D30000B0E04BF09020CF1080C0B0F04BF0901D4
:100D40000CF1040C8B0F04BF89000CF1020CCB0FCB
:100D500004BF49000CF1010CCCF12003A0EB0C0006
:100D600022FA03F302FA0CF241EA030100F1010056
:100D7000704720F07F4C80EA030023F07F47ACEB04
:100D8000070303F57C5300F0004003F1FF032DE956
:100D900080494FEA154B09B44FEA144325EA0B4E3C
:100DA00024EA03480FF2042606EB132749083E788D
:100DB0005FEA320203FB0667C7F5000707FB06F68A
:100DC0004FEA54374FEAD64606F1020607FB066C97
:100DD000CCF1005C4FEA1C472CEA074C07FB06F4F9
:100DE0000CFB06F504EB15464FEA961634BF0020BF
:100DF0004FF000404FEAD13706FB07FC4FEA1C4C8E
:100E00000CFB0BF7D21B03FB0CF761EB07010CFB90
:100E10000EF7B0EB074072EB17420CFB08F734BF3C
:100E2000A2EB0742B2EB074261EB17414FEA0C44D9
:100E30004FEA910706FB07FC4FEA1C4C0CFB0BF733
:100E4000B0EBC74072EB573203FB0CF734BFA2EB99
:100E5000C742B2EBC74261EB57310CFB0EF7B0EB68
:100E6000C70072EB57720CFB08F734BFA2EBC70246
:100E7000B2EBC70261EB5771039F4FEA816141EA10
:100E8000921104EBCC044FEAD1374FEA826206FBA1
:100E900007FC42EA90124FEA80604FEA1C4C0CFBC0
:100EA0000BF7D21B03FB0CF761EB07010CFB0EF7F2
:100EB000B0EB074072EB17420CFB08F734BFA2EB14
:100EC0000742B2EB074261EB17414FEA8C554FEAFC
:100ED000910704EB9C2406FB07FC4FEA1C4C0CFB1F
:100EE0000BF7B0EBC74072EB573203FB0CF734BF84
:100EF000A2EBC742B2EBC74261EB57310CFB0EF7D6
:100F0000B0EBC70072EB57720CFB08F734BFA2EBD3
:100F1000C702B2EBC70261EB577115EB4C254FEAE4
:100F2000816141EA92114FEA82624FEAD13742EA87
:100F3000901206FB07FC44F100044FEA80604FEA80
:100F40001C4C0CFB0BF7D21B03FB0CF761EB0701EE
:100F50000CFB0EF7B0EB074072EB17420CFB08F7E7
:100F600034BFA2EB0742B2EB074261EB174115EB2E
:100F70001C154FEA813141EA92414FEA823242EA3E
:100F800090424FEA80304FEA0C7644F1000448EA80
:100F900003434EEA0B484FF0000EB2EB080C71EB26
:100FA000030724BF624639464EEB0E0E4FF0000B8E
:100FB0000018524149414BEB0B0BB2EB080C71EBA3
:100FC00003077BF1000B24BF624639464EEB0E0E41
:100FD0004FF0000B0018524149414BEB0B0BB2EBA9
:100FE000080C71EB03077BF1000B24BF6246394606
:100FF0004EEB0E0E51EA020718BF46F0010616EB43
:101000000E7655F1000254F1000103D5BDE88901C7
:10101000BDE80088BDE88901BDE80048B619524125
:1010200041EB0101A3F10103704780807F7E7D7C4D
:101030007B7A7978777676757473727171706F6E6A
:101040006E6D6C6C6B6A6A69686867666665646415
:10105000636362616160605F5F5E5E5D5D5C5C5B9F
:101060005B5A5A595958585757565655555554540E
:10107000535352525251515050504F4F4F4E4E4D6C
:101080004D4D4C4C4C4B4B4B4A4A4A4949494848B8
:1010900048474747474646464545454444444443F8
:1010A00043434342424242414141002B9C4630D49B
:1010B00077002BD01CB54FEA370703B44FF0100070
:1010C0004FF01001BAF1000F06D0BCF1000FDCBFE9
:1010D00040F0080040F008014FF000000FBCBDE8F0
:1010E00010400BF1010BBBF1010F08BF5FEA1707BE
:1010F00022BF12F1010211F101014FF0004143F151
:10110000000300F0004043EA00007047F9D357089D
:10111000D0E746EA064613F1400F4FEA16461FDDB8
:1011200013F1200FDFBF16430A46002120335B4234
:10113000BED0C3F1200746EA064602FA07F74FEA97
:10114000164646EA0706C3F1200722FA03F201FA1F
:1011500007F721FA03F14FF0000342EA0702A7E77D
:1011600046EA020646EA06464FEA164646EA0106FF
:10117000BCBF46EA0646360C4FF000034FF00002B3
:101180004FF0000194E72DE9804C9A46934670B4E5
:1011900091E8380007C831EA400C48BF34EA430CF4
:1011A00003D5FFF7E6FDFFF780FFF0BCBDE8008C3C
:1011B0002DE9804C9A46934670B491E8380007C8F0
:1011C00010F0804F08BF13F0804F03D100F005F8F6
:1011D000FFF76BFFF0BCBDE8008C20F07F4780EA92
:1011E000030023F07F4C07EB0C03A3F57C5300F0C6
:1011F0000040A3F1FE0392F0000F00F0B38095F0E1
:10120000000F00F077802DE901494FEA11404FEAC5
:10121000144621EA004800FB06FC24EA064708FBC6
:1012200006F607FB08F800FB07F718EB06484CEB3F
:10123000164C4FEA124B18EB07484FEA15464CEB99
:10124000174022EA0B4E0BFB06FC25EA06470EFB75
:1012500006F607FB0EFE0BFB07F71EEB064E4CEBEC
:10126000164C4FF000061EEB074E4CEB174B18EBDD
:101270000B0840F1000018EB0E0B58EB000840F192
:1012800000008F1A4FF000013CBFC943661B14BF1A
:10129000B5EB040C00213CBFC943F61B4FEA1744D1
:1012A0004EEA8E0E27EA04454FEA1C4704FB07620C
:1012B0002CEA074C05FB07F70CFB05F604FB0CFCBE
:1012C00016EB074642EB174216EB0C4642EB1C426C
:1012D0001BEB060658EB0202414146EA9E0601D589
:1012E000BDE80189B619524141EB0101A3F10103A7
:1012F000BDE801894FEA14454FEA114724EA054643
:1013000021EA074C05FB07F406FB07F70CFB06F187
:1013100005FB0CFC11EB074144EB17444FEA124765
:1013200011EB0C4144EB1C4422EA074C05FB07F28D
:1013300006FB07F70CFB06F605FB0CFC16EB074655
:1013400042EB174216EB0C4642EB1C456A1854F16F
:10135000000148BF7047B619524141EB0101A3F1AA
:101360000103704795F0000F37D04FEA11424FEA62
:10137000144721EA024624EA074C02FB07F106FB68
:1013800007F70CFB06F402FB0CFC14EB074441EBE3
:1013900017414FEA154714EB0C4441EB1C4125EA79
:1013A000074C02FB07F506FB07F70CFB06F602FBF2
:1013B0000CFC16EB074645EB174516EB0C4645EBC8
:1013C0001C42121951F1000148BF7047B619524131
:1013D00041EB0101A3F1010370474FEA14454FEAC5
:1013E000114724EA054621EA074C05FB07F106FBF5
:1013F00007F70CFB06F24FF0000605FB0CFC12EBA6
:10140000074241EB174112EB0C4251EB1C4148BF24
:101410007047921841EB0101A3F1010370470000EE
:1014200010B5084C00221021204600F030FF0220A9
:1014300005F056FD20460122BDE81040102100F0C5
:1014400026BF0000000801402DE9FF41A020012433
:10145000CDE90004DFF84C8003256946039540463A
:1014600000F00CFE01226021404600F010FF4020F9
:101470000026CDE9000669460294404600F0FEFDD4
:1014800010270097CDE901646946074800F0F6FD92
:10149000CDE9007469464046039500F0EFFDBDE8D4
:1014A000FF810000000801400010014010B5084C09
:1014B00000221021204600F0EAFE082005F010FD71
:1014C00020460122BDE81040102100F0E0BE0000DF
:1014D00000080140FEE70000084900B50989814283
:1014E0000AD0A0F57F41FF3906D028B1B12803D03A
:1014F00002F0A0FF002000BD012000BDB0010020CF
:1015000003480021817081638162C1620163704779
:101510005801002010B50F49052808D2DFE800F077
:10152000030514161800812000E091200870C020E7
:10153000487000208870C870064A042105F0FAFC43
:10154000BDE8104005F032B8A120EFE7B120EDE78B
:101550000120EBE798000020014800F097BB000055
:101560009C03002030B590F840500124AC40C56B7E
:101570006C60046863604368102B036803D0996053
:101580000068C26030BD9A600068C16030BD000074
:101590002DE9F05F674C2069002824D166480025BA
:1015A000664F05702078664EF8B121464FF001086D
:1015B000C96B012830D0DFF88CB1DFF88C9102289C
:1015C0003FD003280FD100290DD10121584600F04A
:1015D00051FE022120B15D485D4A006890427DDBEA
:1015E0006163A5702570BDE8F09F0021084606F0F4
:1015F00087FC306847F230518842F4D0012227201E
:10160000316005F0CBF93068012241083960BDE84E
:10161000F05F252005F0C2B90029E4D1A07808B90F
:1016200084F80280607820B1012806D000210846A5
:101630007CE0BDE8F05F06F0F5BABDE8F05F06F0CB
:101640003DB92021434800F015FEDFF80CA1D8B1C8
:101650003E4842490068884227DC10F0FF4F24D002
:10166000C4F83480A5702570E06B0028BBD03C49DD
:10167000212005F073F93A4804F03CFF3949CAF8D3
:1016800000000860E563AEE7E06B58B13449212003
:1016900005F064F9324804F02DFF3249CAF8000021
:1016A0000860E563C4F834809BE701215C46584636
:1016B00000F0E0FD012896D10121204600F0DAFD7E
:1016C000012890D13068494688420DD00122272058
:1016D000316005F063F93068410800E007E001225D
:1016E0002520396005F05AF91F4902201EE001212A
:1016F0005C46584600F0BEFD0128C4D101212046B9
:1017000000F0B8FD0128BED13068494688420BD0B0
:1017100001222720316005F041F93068012241089B
:101720002520396005F03AF90F490120BDE8F05F46
:1017300006F0E6BB5801002090070020AC00002016
:10174000B0000020000C0140C0D40100680000205F
:1017500000C0DA4400100140C400002000007A43B9
:10176000D5000020840000200070170070B5404BA9
:1017700090B01879002878D0022871D2DFE800F004
:1017800070013C4900240C6000F0B4F96A463A4903
:1017900004E00D196D7A1555641CE4B28442F8D347
:1017A00036499DF800001924086035499DF801006C
:1017B000087034499DF8020008709DF80300324912
:1017C0009DF8042002EB002008609DF805002F49D9
:1017D0009DF8062002EB002008609DF807002C49C8
:1017E0009DF8082002EB002008609DF809002949B7
:1017F000401C2B4A08609DF80A5027482749062DAF
:101800002CD2DFE805F02B0309111B240068A0F19E
:10181000700570300D601FE00068A0F1CB04CB3084
:101820000C601060322007E00068A0F29D1400F206
:101830009D100C6010606E2058710FE00068A0F2DF
:10184000FB2400F2FB200C601060D220F4E700685B
:10185000A0F1CB05CB300D6010605C71FFF750FE3E
:1018600010B0BDE8704002F0E5BD10B070BD0000E2
:10187000B0010020840100205407002068010020EE
:1018800058010020590100206C0100207001002047
:10189000740100208C010020540100206001002010
:1018A0006401002070470000F0B52A4C2A4D012643
:1018B000226942B1214602274969491C012A0AD0FE
:1018C000022A39D114E0052804D100216161287071
:1018D0002661E161F0BD616168540229FAD3276194
:1018E000A878697800EB0120E0613B2824D2F0BDA4
:1018F00061613B2920D26854E0698142F7D368795D
:101900000102A8790843FFF7E7FDA8B1E879297A31
:101910004FF2021301EB0020C21A0421984216D0A4
:1019200006DC6FF4704140180AD0C02804D109E0E9
:101930000F2A09D0102A0AD0BDE8F04002F07ABD83
:101940002671F0BD2771F0BD03202071F0BD21711B
:10195000F0BD0000B00100205407002072B6074C13
:101960004FF40065A61400222946204600F08FFCA3
:1019700000223146204600F08AFCF4E700080140CE
:10198000044B0022DA61044A136943F00103136136
:1019900001807047E003002000200240144800222C
:1019A000C168CB06134904D5CA6942F00202CA6174
:1019B0001022C3685B0705D5CB6943F00103CB61F7
:1019C00042F00402C369DB0707D0CB6943F004038C
:1019D000CB61C16921F00101C161A2F580710139BA
:1019E00001D0C2607047C16921F00101C161704737
:1019F00000200240E003002070B5054600F04CFCDA
:101A00000646114C09E0681C07D025B100F044FCE3
:101A1000801BA84201D9032070BDE068C007F2D145
:101A2000E068800601D52020E060E068C00605D4AB
:101A3000E069C00702D1E068400703D5FFF7AEFFB9
:101A4000012070BD002070BD00200240064A002128
:101A5000D16106490A6942F002020A6148610869D7
:101A600040F0400008617047A007002000200240BD
:101A700070B50024FFF74EFDFFF718FD4FF47A769E
:101A8000164D02E0641CB44205D81021284600F02F
:101A9000F1FB0028F6D104F039FD0446FFF7C0FC45
:101AA0000F48210206D501218170E04320F07F44D8
:101AB000641C01E000218170204606F0E1FD094927
:101AC00006F026FE084906F023FE084906F020FE2F
:101AD000BDE87040064906F089BC000000100140D6
:101AE000900000200100A03400007A440020FE4451
:101AF00000801B450448F5228178407802EB0020E5
:101B00000844C0B2704700005407002010B590F898
:101B100021100022022905D00421816380F82020B1
:101B2000012010BD01680B6823F00E030B600168F3
:101B30000B6823F001030B6090F84030C46B012167
:101B400001FA03F3636080F8211080F8202010462A
:101B500010BD00002DE9F05F90F82110002402294B
:101B600003D004218163012485E001680A6822F022
:101B70000E020A6001680A6822F001020A603F4E04
:101B80003E4FB215DFF8F4C0DFF8F090DFF8ECA0BC
:101B9000DFF8E8B0DFF8E4E00168783F13011502F0
:101BA000ACF1640CA9F15009AAF13C0AABF1280B85
:101BB000AEF1140E4FF48018B14227D9B9420ED0BD
:101BC000614512D049451DD0514518D0594518D00E
:101BD000714501D1424615E0294EB14201D10122A1
:101BE00010E0274E1436B14201D110220AE0244EF3
:101BF0002836B14206D0224A3C32914201D11A46DF
:101C000000E02A461E49091F0A602BE0B94213D0A2
:101C1000614517D0494522D051451DD059451DD0A9
:101C2000714501D142461AE0B14202D14FF08072B3
:101C300015E0134EB14201D1012210E0104E1436CE
:101C4000B14201D110220AE00D4E2836B14206D031
:101C50000B4A3C32914201D11A4600E02A4607491C
:101C600080394A60012180F82110002180F820107D
:101C7000416B01B188472046BDE8F09F80000240DB
:101C80000804024090F82100704700002DE9F05F41
:101C9000C16B0A6801680B68046C4FF0040808FA0D
:101CA00004F8844D844E854FDFF814C2DFF8149297
:101CB000DFF814A2DFF814B2DFF814E218EA020F1A
:101CC00065D05FEA437862D50A68920603D40A6851
:101CD00022F004020A60DFF8F0814FF480620168AC
:101CE00008F1140813011402414524D9A9420DD06A
:101CF000B1420FD0B9421AD0614515D0494515D02F
:101D0000514501D1120312E0594501D104220EE0E0
:101D1000714501D140220AE06D4D1435A94206D02B
:101D20006B4A2832914201D11A4600E022466749A7
:101D3000091F0A6029E0A94213D0B14215D0B94267
:101D400020D061451BD049451BD0514502D14FF4ED
:101D5000800217E0414502D14FF0806212E0594500
:101D600001D104220EE0714501D140220AE0584D14
:101D70001435A94206D0564A2832914201D11A465A
:101D800000E022464B4908394A60C16A71E04FF0D1
:101D9000020808FA04F818EA020F70D05FEA8378A4
:101DA0006DD50A68920606D40A6822F00A020A6013
:101DB000012180F82110DFF810814FF400720168D2
:101DC00008F1140813011402414524D9A9420DD089
:101DD000B1420FD0B9421AD0614515D0494515D04E
:101DE000514501D1120312E0594501D102220EE002
:101DF000714501D120220AE0354D1435A94206D0A3
:101E0000334A2832914201D11A4600E022462F4936
:101E1000091F0A6029E0A94213D0B14215D0B94286
:101E200020D061451BD049451BD0514502D14FF40C
:101E3000001217E0414502D14FF0007212E05945FF
:101E400001D102220EE0714501D120220AE0204D8D
:101E50001435A94206D01E4A2832914201D11A46B1
:101E600000E02246134908394A60002180F820101A
:101E7000816A00291CD0BDE8F05F0847FFE708250C
:101E8000A540154214D01A0712D50A6822F00E0296
:101E90000A6090F84020C36B012101FA02F25A60F7
:101EA000816380F82110002180F82010016BE0E7A9
:101EB000BDE8F09F080002401C00024030000240D4
:101EC00044000240580002406C00024008040240F6
:101ED0001C04024030B560B11A4B026814219A42CA
:101EE00009D2194B1344B3FBF1F18900016417497E
:101EF0000AE0012030BD134B5B421344B3FBF1F108
:101F0000890001640F490839C163022180F821105A
:101F1000136843F6F0718B43F0E901142143D0E9D3
:101F200002452C43214304692143446921438469C8
:101F30002143194311600021416301224277017757
:101F4000084630BD08040240F8FFFDBF0000024013
:101F500070B5044690F82000002501280CD001201F
:101F600084F8200094F821600020012E06D084F827
:101F700020000225284670BD022070BD022684F88C
:101F80002160A0632068066826F0010606602046EE
:101F9000FFF7E8FAE06A00282068016802D041F003
:101FA0000E0106E021F0040101602068016841F0A3
:101FB0000A0101602068016841F001010160D9E770
:101FC0000348016941F08001016100207047000071
:101FD000002002402DE9F05F07461C488846002497
:101FE000017E15461E46012909D001218146017650
:101FF0004CF2503A5046FFF7FFFC18B122E00220A5
:10200000BDE8F09F012F02D0022F00D00427D34655
:10201000DFF83CA0220128463146FEF727F981B2BD
:1020200008EB4400FFF7ACFC5846FFF7E5FCDAF894
:10203000102022F00102CAF8102018B9641CE4B282
:10204000BC42E7D3002289F81820D9E7E00300203A
:1020500000200240064900200A69120607D5054AF9
:102060004A60054A4A600969090600D5012070479F
:102070000020024023016745AB89EFCD2DE9F84FE1
:10208000DFF8C8910024A9F1040B23460F2709F1BA
:10209000040AABF1040ED1E00125A54006EA0502D1
:1020A000AA4276D1DFF8A8C14E68A6EB0C086645B7
:1020B0002BD00DDC032E34D005DC36B3012E19D025
:1020C000022E2FD11BE0112E16D0122E2AD119E08C
:1020D000B8F5881F19D006DCB8F5803F15D0B8F5E3
:1020E000801F1FD111E0B8F5001F0ED0B8F5041FF6
:1020F00018D10AE0CB6815E0CB681B1D12E0CB6855
:1021000008330FE0CB680C330CE08B682BB1012B4C
:102110004FF0080303D0456104E0042302E00561A9
:1021200000E00023FF2A01D8064601E000F1040682
:102130004FEA840501D9A5F12005D6F8008007FAF9
:1021400005FC28EA0C0803FA05F548EA0508C6F874
:1021500000804D68ED0070D53E4DAE6946F0010639
:10216000AE61AD6924F0030605F0010500953A4D16
:1021700006EB050CDCF80850A607360F07FA06F840
:1021800025EA0805DFF8D480404503D14FF0000868
:1021900025E052E0DFF8C880404502D14FF0010849
:1021A0001DE0DFF8C080404502D14FF0020816E084
:1021B000DFF8B480404502D14FF003080FE0DFF8AC
:1021C000AC80404502D14FF0040808E0DFF8A08061
:1021D000404502D14FF0050801E04FF0060808FA2B
:1021E00006F848EA0508CCF808804D68D9F8006080
:1021F000ED024D4601D5164300E096432E604D6832
:10220000DAF80060AD02554601D5164300E096436A
:102210002E604D68DBF80060AD035D4601D51643C6
:1022200000E096432E604D68DEF80060ED037546D1
:1022300001D5164300E096432E60641C0A681646DA
:10224000E2407FF429AFBDE8F88F000008040140A8
:102250000000111000100240000001400008014081
:10226000000C014000100140001401400018014022
:10227000001C01408068084000D001207047C268FF
:1022800021EA02030A4043EA0241016170470AB1B0
:10229000016170470904FBE701488068704700004E
:1022A00054000020704770472DE9F0410168044652
:1022B0004A694E6890F83E000025D743FA050BD4D2
:1022C000F243D20508D46FF4807201254A61216877
:1022D0000A6842F400420A60B90508D4F143C9050E
:1022E00005D422686FF4007145F00205516179054B
:1022F00025D4F143C90522D4638D94F83D10226B97
:10230000202808D13BB9212910D029290ED028290D
:1023100001D1212A0AD022686FF48061516145F011
:102320000405102806D0402804D008E0204601F01B
:102330008BFF04E02068016841F4007101603805FA
:1023400008D4F043C00505D421686FF4006045F05F
:1023500008054861002D07D0206C284320642046E2
:10236000BDE8F04101F0DEBBBDE8F0812DE9F047AA
:10237000026800215368C66A90F83E4090F83D50CC
:10238000102C12D0402C10D0046C002C7DD054693D
:10239000E443A6077AD4DE43B60577D4036C03B1D1
:1023A0009169BDE8F04701F02BBF976951694FF47F
:1023B0002A0CC9435FEAC1784FF02A4904D0664528
:1023C0002AD04E4528D010E0DE43B6050DD4C16AB0
:1023D000614501D1012103E0C16A494501D10821CC
:1023E000C162BDE8F04701F071BE0E0716D4DE43AE
:1023F000B60513D4416CC9B21161416B09B1896A48
:1024000029B9816B002907D0896A002904D00068A6
:10241000416841F400614160BDE8F0878E0706D451
:10242000DE43B60503D4BDE8F04701F0A3BDFE438B
:10243000526876074FEA02521DD4002AECDB0A06E6
:1024400008D4DA43520505D4490705D5BDE8F0475D
:1024500001F034BD4907DFD4D9438905DCD4212DEF
:1024600005D0402CD8D1BDE8F04701F075BEBDE8DD
:10247000F04701F0E1BC002ACEDB4A060BD4DA4378
:10248000520508D4490708D501E00DE00EE0BDE88B
:10249000F04701F05DBC4907BED4D9438905BBD4E0
:1024A000BDE8F04701F0EABB916970E7E10606D4A8
:1024B000D943890503D4BDE8F04701F00DBF2821B9
:1024C000212D27D0292D25D0650655D4DD436D0556
:1024D00052D4640752D590F83D30448D002C9BD0E7
:1024E0001269446A2270426A521C4262428D521E34
:1024F0004285428D002A8FD12A2B8DD102685368E4
:1025000023F4806353602222026380F83D1000F0C0
:1025100057F981E7250623D4DD436D0520D46407F0
:1025200020D590F83D30448D002CF2D0446A2478B8
:102530001461426A521C4262428D521E4285428D93
:10254000002AE6D1292BE4D10268536823F4806382
:1025500053602122026380F83D1000F032F95BE7FE
:102560006107D6D4D9438905D3D4418D0029D0D071
:10257000416A097811610AE06107CAD4D943890523
:10258000C7D4418D0029C4D01169426A1170416AD3
:10259000491C4162418D491E41853DE7704700005D
:1025A00070B5040025D094F83D00002520B984F8CA
:1025B0003C50204600F0BEF8242084F83D002068FE
:1025C000016821F0010101602068016841F40041C7
:1025D00001602068016821F40041016000F020FAE8
:1025E0004D4A6168914201D84C4900E04C4988420B
:1025F00001D2012070BD4B492368B0FBF1F15E6848
:1026000026F03F060E435E606368934206D94FF49E
:10261000967359434FF47A73B1FBF3F12368491C65
:102620001E6A26F03F06314319626168914210D854
:102630004900401EB0FBF1F2521CC2F30B02042A07
:1026400001D2042022E0B0FBF1F0401CC0F30B00EB
:102650001CE0A268F2B301EBC10303EB0116431EB9
:10266000B3FBF6F35B1C43F480431B0549D092B3E4
:1026700001EBC10202EB0111401EB0FBF1F0401C66
:10268000C0F30B0040F4804040F400402168CA6968
:102690004CF6FF739A431043C861D4E90710014315
:1026A0002068026822F0C00211430160D4E90301EE
:1026B00001432068826848F2FF339A4311438160E6
:1026C000D4E9050108432168CA6822F0FF021043DB
:1026D000C86001E00EE016E02068016841F00101E9
:1026E00001602564202084F83D00256384F83E5075
:1026F000002070BD01EB4106431EB3FBF6F35B1CEB
:10270000B3E70120C2E701EB4101401EB0FBF1F04D
:10271000401CC0F30B00B7E7A086010080841E00B8
:1027200000093D0040420F007047704770477047F6
:102730007047000010B586B0002100910191029110
:10274000039100681A49884230D11A4CA06940F0C0
:102750000800A061A069694600F008000490C0204C
:10276000009012200190032003901348FFF786FC8D
:10277000E06940F40010E061E069002200F400101C
:10278000049011461F2000F083F81F2000F072F81B
:1027900000221146202000F07BF8202000F06AF88B
:1027A00006480068416841F4E061416006B010BD30
:1027B0000054004000100240000C0140D0010020F5
:1027C0007047704702488168027811448160704701
:1027D00054000020074810B5016841F01001016065
:1027E000032000F075F8002000F006F800F024F84F
:1027F000002010BD0020024070B50D4D04464FF47E
:102800007A712878B1FBF0F00A490968B1FBF0F061
:1028100000F0F2FB48B9102C07D200222146501ECE
:1028200000F036F800206C6070BD012070BD000023
:1028300054000020600000200C4808B5816941F078
:1028400001018161816901F001010091C16941F0DB
:102850008051C161C06900F0805000900448416817
:1028600021F0E06141F00071416008BD00100240BC
:1028700000000140002809DB00F01F020121914007
:102880004009800000F1E020C0F80011704700000E
:10289000F0B40E4B1B680C46C3F30223C3F10705CB
:1028A000042D00D90425191D072901D2002300E0B9
:1028B000DB1E012606FA05F1491E214099409E4083
:1028C000761E16403143F0BC04F0D4BB0CED00E0A2
:1028D000064900F0070208684FF6FF03184040EA77
:1028E0000220034A10430860704700000CED00E02E
:1028F0000000FA052DE9F0470F46050061D0434E70
:10290000306800F00700B84209D2306820F00700B4
:1029100038433060306800F00700B84251D1286871
:102920003B4C810712D5400703D5606840F4E06056
:1029300060602878000703D5606840F460506060EC
:102940006068A96820F0F000084360602878C0073C
:1029500028D06868012810D02168022810D0890783
:1029600000292EDA616821F0030101436160FFF75D
:1029700093FC804641F288390DE021688903EFE736
:102980008901EDE7FFF788FCA0EB0801494502D972
:102990000320BDE8F0876068696800F00C00B0EBC8
:1029A000810FEFD1306800F00700B8420BD93068D2
:1029B00020F0070038433060306800F00700B8426C
:1029C00001D00120E5E72878400705D56068E9686F
:1029D00020F4E060084360602878000706D560684E
:1029E000296920F4605040EAC100606000F038F8C6
:1029F0006168084AC1F30311515CC8400649086088
:102A000006480068FFF7F8FE0020C2E700200240F9
:102A100000100240EC8A00086000002058000020EE
:102A20000448054900684968044AC1F30221515C21
:102A3000C84070476000002000100240FC8A000877
:102A40000448054900684968044AC1F3C221515C41
:102A5000C84070476000002000100240FC8A000857
:102A60000E4A51680E4801F00C03042B11D0082BBC
:102A70000FD10C48C1F38343C903C05C0AD5516828
:102A8000084AC1F34041921E515C054A5043B0FBD5
:102A9000F1F07047044948437047000000100240BD
:102AA00000127A00DC8A000800093D002DE9F84F89
:102AB000040070D02078C04DC00749D06868C0F3CA
:102AC0008100012807D06868C0F38100022809D17D
:102AD0006868C00306D52868800339D56068002877
:102AE000E7D035E06068B0F5803F0BD010B1B0F5AD
:102AF000A02F11D0286820F480302860286820F4A6
:102B0000802002E0286840F480302860606890B13E
:102B1000FFF7C2FB06460AE0286840F480202860E0
:102B2000F0E700BFFFF7B8FB801B642873D8286864
:102B30008003F7D50CE0FFF7AFFB064605E000BFCA
:102B4000FFF7AAFB801B6428F0D828688003F7D41D
:102B500020789A4E80074FF001094FF0000839D5D0
:102B6000686810F00C0F07D06868C0F38100022875
:102B700009D16868C00306D42868800714D5206985
:102B8000012808D110E02069B0B1C6F80090FFF725
:102B900083FB074605E00AE1FFF77EFBC01B022826
:102BA000C4D828688007F7D52868616920F0F80044
:102BB00040EAC10028600DE0C6F80080FFF76CFB1A
:102BC000074604E0FFF768FBC01B022823D82868EB
:102BD0008007F7D4207800072CD57948A169D9B1AE
:102BE000C0F80090FFF758FB074604E0FFF754FBDE
:102BF000C01B02280FD8686A8007F7D571484FF4C8
:102C0000FA510068B0FBF1F0009000BF0098411E3F
:102C10000091FAD20EE080E0C0F80080FFF73CFBA4
:102C2000074604E0FFF738FBC01B022875D8686A26
:102C30008007F7D42078400760D5E8690027C000F6
:102C400008D4E86940F08050E861E869012700F0A5
:102C5000805000905C480168C90513D40168834620
:102C600041F480710160FFF717FB824606E000BF68
:102C7000FFF712FBA0EB0A0064284ED8DBF8000037
:102C8000C005F5D5E06801280AD008B1052813D0A1
:102C9000286A20F001002862286A20F0040002E07F
:102CA000286A40F001002862E06841F2883B98B150
:102CB000FFF7F2FA82460BE0286A40F0040028622F
:102CC000EEE700BFFFF7E8FAA0EB0A0159455AD832
:102CD000286A8007F6D50CE0FFF7DEFA824605E0A9
:102CE000FFF7DAFAA0EB0A0159454CD8286A8007A9
:102CF000F6D41FB1E86920F08050E861E06988B33C
:102D00006968C1F38101022944D00228C6F86080B5
:102D100004D0FFF7C1FA044638E034E0FFF7BCFA0C
:102D2000074604E0FFF7B8FAC01B02282BD8286832
:102D30008001F7D4206AB0F5803F05D16868A168AA
:102D400020F4003008436860D4E90801084369684A
:102D500021F4741108436860C6F86090FFF79CFA8C
:102D6000044606E025E000BFFFF796FA001B0228A4
:102D700009D828688001F7D51BE000BFFFF78CFA5F
:102D8000001B022802D90320BDE8F88F28688001C3
:102D9000F4D40EE00128F7D06868226A00F480318C
:102DA000914204D1616A00F47010884201D0012080
:102DB000EAE70020E8E7000000100240000042427D
:102DC0008004424260000020007000407047000014
:102DD00038B50446006842688168C9434B0606D589
:102DE000CB0704D1D3435B0601D4216C05E08B07EC
:102DF00008D4D3431B0605D4616C01B02046BDE85E
:102E0000304008478B0601D54B0646D4D3439B067A
:102E100043D44B060AD494F85130032B3ED0636D53
:102E200043F004036365C36883680093890609D48B
:102E3000616D41F00101616581680091016821F0D7
:102E400040010160606D002827D02068416821F0B2
:102E5000E0014160012084F85100900722D02068F1
:102E6000416821F003014160104DE06C40B14563C1
:102E7000E06CFEF76FFE18B1606D40F040006065D9
:102E8000A06C002809D04563A06CFEF763FE002803
:102E900003D0606D40F04000606538BDC168806857
:102EA000009038BD2046FFF791FF38BDF16500085E
:102EB00070B5040009D0606A002540B125616561E4
:102EC000A56294F8510040B10CE0012070BD60682B
:102ED000B0F5827FF4D0E561F2E784F850502046E7
:102EE00000F040F8022084F851002068016821F0C9
:102EF00040010160A088218900F4827001F404413E
:102F00000843A18901F400610843217C01F002011A
:102F10000843217D01F001010843218B01F4007178
:102F20000843217F01F03801084394F8201001F094
:102F300080010843218D01F4005108432168086095
:102F4000A069042101EA1040216848602068C16935
:102F500021F40061C1616565012084F85100002001
:102F600070BD000030B585B0002400940194029437
:102F7000039400681C49884233D11C48C16941F45C
:102F80008041C161C16901F480410491816941F0CE
:102F9000080181618069164D00F0080004904FF42B
:102FA00020400090022001900320039069462846AB
:102FB000FFF764F84FF48040CDE9000469462846E5
:102FC0000294FFF75BF8002211462420FFF760FC13
:102FD0002420FFF74FFC07480068416841F0A0013A
:102FE000416005B030BD00000038004000100240D4
:102FF000000C01402402002010B5401EB0F1807F7B
:1030000001D3012010BD4FF0E02460610F21601753
:1030100004F030F80020A06107202061002010BDDE
:103020007047704770B590F83C20012A2CD00124DD
:1030300080F83C40022280F83D2003685A689D6871
:1030400022F070060A6832435A60104B02689A42B6
:103050000ED00F4B9A420BD0B2F1804F08D00D4BDF
:103060009A4205D00C4B9A4202D00C4B9A4204D1A2
:10307000496825F080031943916080F83D400021A4
:1030800080F83C10084670BD022070BD002C014045
:10309000003401400004004000080040000C0040E3
:1030A00010B5040003D094F83D0010B107E00120F2
:1030B00010BD002084F83C00204600F01FF80220DC
:1030C00084F83D00211D206803F0A4FB012084F852
:1030D000460084F83E0084F83F0084F8400084F8FD
:1030E000410084F8420084F8430084F8440084F8E6
:1030F000450084F83D00002010BD000008B50068C0
:103100000B49884212D10B48816941F40061816109
:103110008069002200F40060009011461920FFF73A
:10312000B7FBBDE808401920FFF7A4BB08BD0000AD
:10313000002C01400010024090F83D10012901D000
:1031400001207047022180F83D100168CA6842F0F2
:103150000102CA6000680E4988420ED00D498842BB
:103160000BD0B0F1804F08D00B49884205D00B49F5
:10317000884202D00A49884204D1816801F00701DF
:10318000062903D0016841F0010101600020704769
:10319000002C0140003401400004004000080040C1
:1031A000000C004070B5044690F83C000025012852
:1031B00017D0012684F83C60022084F83D00206886
:1031C000826822F0770222F47F42826008685028E9
:1031D00038D00DDC20284FD005DC90B3102811D159
:1031E0004AE0022070BD302846D040280AD13BE09A
:1031F00060282FD070280DD0B0F5805F03D0B0F5D7
:10320000005F12D0012584F83D60002084F83C0066
:10321000284670BDCB68D1E90121206803F040FB4E
:103220002068816841F0770109E0CB68D1E901218C
:10323000206803F035FB2068816841F4804181609B
:10324000E1E719E0CA684968206803F03BFB5021B8
:10325000206806E0CA684968206803F044FB6021E2
:10326000206803F027FBCEE7CA684968206803F0AE
:1032700029FB40212068F4E7226801461046F0E768
:10328000704770B50446006801694FF00005C943F6
:10329000890715D4C168C943890711D4E91E0161A2
:1032A00001202077206880698007204602D0FFF740
:1032B000E7FF04E000F098F8204600F096F8257744
:1032C00020680169C943490717D4C168C943490740
:1032D00013D46FF004010161022020772068806917
:1032E00010F4407F204602D0FFF7CAFF04E000F050
:1032F0007BF8204600F079F8257720680169C943FA
:10330000090716D4C168C943090712D46FF0080130
:103310000161042020772068C0698007204602D020
:10332000FFF7AEFF04E000F05FF8204600F05DF824
:10333000257720680169C943C90617D4C168C94304
:10334000C90613D46FF010010161082020772068AE
:10335000C06910F4407F204602D0FFF791FF04E0DF
:1033600000F042F8204600F040F825772068016917
:10337000C943C90708D1C168C943C90704D1891E17
:103380000161204600F032F820680169C94309064E
:1033900009D4C168C943090605D46FF080010161F1
:1033A0002046FFF73DFE20680169C943490609D45C
:1033B000C168C943490605D46FF040010161204648
:1033C00000F09CF820680169C94389060BD4C168E4
:1033D000C943890607D46FF0200101612046BDE88A
:1033E0007040FFF71EBE70BD70477047414930B452
:1033F00088427CD140484168012901DA012200E07D
:103400000022491C4A4301214260012A00D1816007
:10341000C368C82B01DA012200E000225B1C5A437A
:10342000C260022A00D101614269052A01DA012342
:1034300000E00023521C53434361052B00D18161FE
:10344000C3690A2B01DA012200E000225B1C5A4307
:10345000C2610A2A00D10162426A322A01DA0123DA
:1034600000E00023521C53434362322B00D181629F
:10347000C26A642A01DA012300E00023521C53438C
:10348000C362642B00D10163436B4FF4FA74A3420F
:1034900001DA012200E000225B1C5A434263A2428F
:1034A00000D18163C26B4FF47A74A24201DA012326
:1034B00000E00023521C5343C363A34200D10164C4
:1034C000426C41F288318A4201DA012300E0002394
:1034D000521C534343648B4203D1816C21B10021C0
:1034E000816430BC00F0BCBF0121F9E7FFE730BCCC
:1034F000704700007C02002000000020704738B5B3
:10350000044690F84200202801D0022038BD61B165
:103510005AB10120206300206063204603F050FC74
:103520000028F3D1216B012901D0012038BD216889
:103530000A684968009121680C3151E8002F42F077
:10354000100241E80023002BF5D138BD70477047C9
:10355000F8B5016804460868CA684B6910F00F0F97
:103560004FF0000559D003F0010602F4907737437D
:1035700065D0C10705D0D10503D5616C41F00101CB
:103580006164410705D5D90703D0616C41F00201A0
:103590006164810705D5D90703D0616C41F004014E
:1035A0006164010707D502F02001314303D0616C4B
:1035B00041F008016164616C00293AD0800604D5AD
:1035C000900602D5204603F03DFB20684069616CFF
:1035D000C0F38010090700D460B3204603F0FDFA61
:1035E00020684069400621D52068143050E8001F4B
:1035F00021F0400140E80012002AF5D1E06BA8B1AB
:103600006D494163E06BFEF7A5FA002811D0E06B2D
:10361000416B01B0BDE8F040084783060FD5930623
:103620000DD52046BDE8F84003F00CBB2046FFF75F
:103630008EFFF8BD2046FFF78AFF6564F8BD266B54
:103640002023012E7CD1C6067AD5D60678D5086807
:103650004868009048694FF00206400640D5E16B8B
:10366000086840680004000CE8D0A28D8242E5D9C9
:10367000E085886920282DD020680C3050E8001F94
:1036800021F4807140E80012002AF5D1206814303E
:1036900050E8001F21F0010140E80012002AF5D196
:1036A0002068143050E8001F21F0400140E800126B
:1036B000002AF5D184F84230256320680C3050E8A8
:1036C000001F21F0100140E80012002AF5D1E06B44
:1036D000FEF71CFA6663A08DE18D401A81B22AE0E4
:1036E000A08DE18D401A81B2E08D0028A6D000297E
:1036F000A4D022680C3252E8000F20F4907042E807
:103700000007002FF5D12068143050E8002F22F078
:10371000010240E80027002FF5D184F842302563EC
:1037200020680C3050E8002F22F0100240E80023FF
:10373000002BF5D166632046FFF708FFF8BDFFE7D1
:1037400005062BD5150629D594F841002128F5D179
:10375000A068B0F5805F01D12069B0B1206A411C3A
:103760002162216800784860E08C401E0004000C53
:10377000E084E3D12068C16821F08001C160206845
:10378000C16841F04001C160D8E7206A0088C0F3F9
:1037900008004860206A801C2062E5E74006CDD51D
:1037A0005006CBD5CA68204622F04002CA6084F891
:1037B000413000F015F9C1E7DD6A000870B504007A
:1037C00004D094F84100002510B106E0012070BD3E
:1037D00084F84050204600F023F8242084F841006B
:1037E0002068C16821F40051C160204603F08CFAC2
:1037F0002068016921F4904101612068416921F04C
:103800002A0141612068C16841F40051C1606564CA
:10381000202084F8410084F842006563002070BDD8
:10382000F0B585B0002400940194029403940546F9
:1038300003685648DFF850C102210322544E071591
:10384000634528D1836943F480438361836903F42A
:1038500080430493836943F0040383618069039286
:1038600000F0040004900802CDE9000169463046EA
:10387000FEF704FCCDE90074694630460294FEF779
:10388000FDFB002211462520FFF702F82520FEF758
:10389000F1FF404842E0DFF800C1634545D1C3690C
:1038A00043F40033C361C36903F4003304938369B1
:1038B00043F0040383618069039200F004000490E4
:1038C0000420CDE9000169463046FEF7D7FB082009
:1038D000CDE90004694630460294FEF7CFFB2D4E39
:1038E0002E48D836C6E900048020C6E902402020D0
:1038F0003461C6E905403046F461FEF7EBFA08B1E1
:10390000FEF72CF8EE630022114626207562FEF7C2
:10391000BFFF2620FEF7AEFF1E4848300068C16892
:1039200041F06001C16005B0F0BD1D4DAB42FAD160
:10393000C36943F48023C361C36903F48023049300
:10394000836943F0080383618069CDE9007100F069
:103950000800CDE90320134D69462846FEF78EFB8B
:10396000E814CDE90004694628460294FEF786FB78
:10397000002211462720FEF78BFF2720FEF77AFF53
:1039800004489030CAE700000038014000100240AF
:1039900000080140C4020020004400406C000240C6
:1039A00000480040000C01407047704790F84130DB
:1039B000202B01D00220704779B172B1016282845C
:1039C000C28400214164212180F841100068C1684F
:1039D00041F08001C1600020704701207047000065
:1039E00000680449884204D1002202210248FEF7FF
:1039F0004EBC704700440040000801400D4800687C
:103A0000C00700D000BE00250B4E0C4C4FF40067E1
:103A10004FF480580021084604F072FA35700022F5
:103A200039462046FEF733FC002241462046FEF789
:103A30002EFCEFE7F0ED00E0580100200008014007
:103A40000148FEF731BC0000D00100200148FEF71C
:103A50008DBC0000D001002038B5406A002190F8EC
:103A60003D202B4B46F2A8141B68B3FBF4F3C3EBC9
:103A7000C30303EB830300933BB15B1E0093036816
:103A80001B689B0505D5009BF6E7036C43F02003FC
:103A90000364436B03B19962836B03B1996203685A
:103AA0001C6824F480641C604185436B03B1596336
:103AB000836B03B1596303681C6824F001041C6024
:103AC00090F83D402023602C0BD0282434EA0202D9
:103AD0000FD080F83D3080F83E1000BFFEF75EFD4D
:103AE00038BD80F83D3080F83E100164FEF7DAFB07
:103AF00038BD0268136843F001031360026813685D
:103B000043F480631360016380F83D40E6E7000002
:103B10006000002000684169C943090601D4002102
:103B20000161704770B5044690F83D0094F83E106E
:103B3000102901D0402906D1222804D121680A6821
:103B400022F400620A60282131EA00024FF00005E9
:103B50004FF0200626D021684968090505D4602861
:103B600003D084F83D6084F83E50256320684168A6
:103B7000090537D5416821F400614160606B90F818
:103B800021203C49012A11D04163606BFDF7E2FF1F
:103B900038B32068016821F00101016084F83D60BC
:103BA000606B1CE0256384F83D10DFE7A06B416388
:103BB000A06BFDF7CFFFA0B120684169C94349065A
:103BC00005D40069616A0870606A401C6062206800
:103BD000016821F00101016084F83D60A06B416B38
:103BE000884710E094F83D10602910D04169C9431E
:103BF000490605D40069616A0870606A401C606209
:103C00002046FEF7CBFC206CC1071CD115E084F8E0
:103C10003D6025644169C943490605D40069616A6C
:103C20000870606A401C60622068016821F0010130
:103C300001602046FEF736FBE5E7810703D4410724
:103C400001D4000704D52068416821F4E061416097
:103C500094F83D00216C49070BD5282809D1064866
:103C6000E062256384F83D6084F83E502046FEF70C
:103C70005BFD70BD593A00080000FFFF10B5C26A35
:103C8000438D0168042B06D0438D032B08D0438D50
:103C9000022B1DD012E04A6822F480624A600CE0D8
:103CA0004B6823F480634B60042A06D0022A04D0B8
:103CB00001680A6822F480620A6001680969426A40
:103CC0001170416A491C4162418D491E418510BDF8
:103CD000012A30D0102A2ED0042A30D0022A2ED029
:103CE0000A6842F400720A6001680969426A117048
:103CF000416A491C4162428D521E42850268126926
:103D00000A70416A491C4162418D491E4185016822
:103D10004A6822F440724A60202180F83D1090F8F1
:103D20003E200021402A80F83E100CD01221016371
:103D3000FEF7FBFC10BD0A6822F48062D3E70A6834
:103D400042F48062CFE70163FEF7F1FC10BD000092
:103D500038B590F83D1022290FD1418D03290DD996
:103D600001680969426A1170416A491C4162418DCA
:103D7000491E4185418D032906D038BDC26A022AF9
:103D800002D0012906D029B10068416821F4806180
:103D9000416038BD274946F2A81300220968B1FBEB
:103DA000F3F101EB8101009101682023009C641E66
:103DB000009422D00C68A405F8D40C6824F4806424
:103DC0000C6001684C6824F4E0644C600168096987
:103DD000446A2170416A491C4162418D491E4185F6
:103DE00080F83D3090F83E1080F83E2040291DD0EC
:103DF00012210163FEF799FC38BD046C44F02004E5
:103E000004644C6824F4E0644C6001680969446A05
:103E10002170416A491C4162418D491E418580F8EB
:103E20003D3080F83E20FEF7B9FB38BD0263FEF757
:103E30007EFC38BD6000002010B5C26A90F83D10CD
:103E400021290BD1418D51B1416A02680978116174
:103E5000416A491C4162418D491E418510BD2023A4
:103E60000021082A13D0202A11D012F5803F0ED04D
:103E70000268546824F4E06454601122026380F8FC
:103E80003E1080F83D3000BFFEF750FC10BD0268C8
:103E9000546824F4E06454600268146844F40074C4
:103EA0001460016380F83D3090F83E2080F83E10A9
:103EB000402AE9D1FEF73CFC10BD000010B590F897
:103EC0003D1090F83E30C26A048DB4B1212903D070
:103ED000402B11D122290FD1418DE1B390F83E1032
:103EE000402942D0416A026809781161416A491C3F
:103EF0004162418D491E418510BD2129E8D1202311
:103F00000021082A13D0202A11D012F5803F0ED0AC
:103F10000268546824F4E06454601122026380F85B
:103F20003E1080F83D3000BFFEF700FC10BD026877
:103F3000546824F4E06454600268146844F4007423
:103F40001460016380F83D3090F83E2080F83E1008
:103F5000402AE9D100E002E0FEF7EAFB10BD00686C
:103F6000416821F48061416010BDBDE8104000F05F
:103F7000F3B8000078B590F83E50C26A046B90F830
:103F80003D6000230168222E73D1066D0EB9402DCD
:103F90006FD0056D1DB90569B5F5404F1BD0458D36
:103FA00095B3468D484D012E20D0448D022C4DD026
:103FB0000C6844F480640C6001684C68240579D571
:103FC000AA4273D0012A71D0082A6FD0102A6DD06E
:103FD000202A6BD06EE04A698A6900920A6842F42E
:103FE00080720A60016D491C016578BDAA4214D136
:103FF0000A6822F480620A6001684A68120504D5E2
:104000000A6822F4806217E0FFE74A698A69009231
:104010000A6842F400720A6050E0082A10D0202A90
:104020000ED0122C0AD0042A03D0022A01D0102A62
:10403000E6D10A6842F480620A603BE0012ADFD0E0
:104040000A6822F480620A600168DEE7042A11D05F
:10405000022A0FD0102A0DD00C6844F400640C60C2
:1040600001684C698C6900940C6824F480640C60CD
:1040700008E025E00C6844F480640C6001684C6939
:104080008969009101684C68240517D5AA4207D0B8
:10409000012A05D0082A03D0102A01D0202A0DD1E8
:1040A0004A6842F480524A6008E0FFE74A6842F4F6
:1040B00080524A6001684A6989690091036578BD48
:1040C00048698869009078BD0000FFFF90F83E10B5
:1040D000402910D00169B1F5804F19D0016DA9B305
:1040E000016D012910D1416C5FF0F10201F44071C2
:1040F00042EAD11106E0016D0029416C05D0C9B238
:1041000041F0010100680161704701F0FE01F9E72B
:1041100090F83D102129416C09D0C9B241F001014C
:1041200002681161416B29B1896A49B902E001F065
:10413000FE01F5E7816B0029E6D0896A0029E3D00A
:104140000068416841F4006141607047FFE7416CDD
:10415000F02201F44071CBE710B590F83D10026DEC
:104160004AB1026D012A14D0026D022A16D0BDE8B0
:104170001040FFF7CFBCC16C0129816C02D0C1F3A4
:10418000072108E00268C9B21161016D891C01654F
:1041900010BD816CC9B20268116123E022291CD0D4
:1041A000428D0AB1212920D0428D002AF0D1212947
:1041B000EED101684A6822F4E0624A6001680A6848
:1041C00042F400720A6000210163202280F83D2041
:1041D00080F83E10FEF7ACFA10BD01680A6842F4A0
:1041E00080720A60016D491CD1E7416A0268097852
:1041F0001161416A491C4162418D491E418510BDD2
:1042000038B50C4690F83D200021282595430268DA
:104210000B4605D051699169009180F83C3038BD5A
:10422000556825F480655560E243540700D50121A7
:10423000120601D5828900E0028B80F83C3092B2F0
:10424000FEF731F838BD00002DE9F04190F83D301F
:104250000446C26A002120261E4F00686FF4806564
:10426000082A01D0202A01D1282B04D0212B17D0D5
:104270004561BDE8F081E762426822F4E062426095
:10428000206845612068026822F480620260216330
:1042900084F83D6084F83E102046FEF745FAE8E7D2
:1042A000E7622122226384F83D6084F83E10416871
:1042B00021F4E0614160206845612068016821F4D3
:1042C000806101602046FFF725FC2046FEF779FA61
:1042D000CFE700000000FFFFF8B590F83D6004460E
:1042E0000068416821F4E06141602068002541696F
:1042F0000091016841F0010101602068016821F42A
:104300008061016020684168090520D5474F222E51
:1043100048D02A2E46D0616B096849686185618D55
:1043200019B1216C41F004012164416821F400615C
:104330004160606BFDF7A6FC012808D0606B476305
:10434000606BFDF707FC10B1606B416B8847608DB7
:1043500008B320684169C943490708D40069616A04
:104360000870606A401C6062608D401E6085206835
:104370004169C943490608D40069616A0870606AE6
:10438000401C6062608D401E6085608D18B1206C9D
:1043900040F004002064206C00B32046BDE8F840E3
:1043A000FFF7C0BBA16B096849686185618D19B1D0
:1043B000216C41F004012164416821F400614160F5
:1043C000A06BFDF75FFC0128C1D0A06B4763A06B19
:1043D000FDF7C0FB0028BAD0A06BB6E72A2E06D1A5
:1043E0002563282084F83D002046FEF7E9F994F87B
:1043F0003D10202028290DD0216B222901D0222E0A
:1044000007D1256384F83D0084F83E502046FEF72E
:10441000D7F9F8BD0649E162256384F83D0084F8C8
:104420003E502046FEF780F9F8BD0000593A0008DA
:104430000000FFFF08490020084B0871486108612F
:10444000C86148708870C860024688611A54401C70
:104450003C28FBD38A617047B0010020540700203C
:1044600070B504211C48FDF705FF1C4C4FF480512A
:1044700020701B48FDF7FEFE60704FF400411948A4
:10448000FDF7F8FE211FA07008780023032800D351
:104490000B700878114A245CD21E0CB9155C1DB152
:1044A000155C022D0DD00FE00F4C54F820506D1C00
:1044B00044F82050052D07D944F820300124145425
:1044C00002E0012C00D11354401CC0B20870032834
:1044D00000D30B7070BD0000001401408D0000205F
:1044E00000100140000801400004002070B50024C5
:1044F0004FF40065134E04E0641CE4B2012002F0A6
:10450000B3FE29463046FDF7B5FE012803D0C82C7E
:1045100010D2002407E0C82CEED30BE0641CE4B2F8
:10452000012002F0A1FE29463046FDF7A3FE18B196
:10453000F02C04D3012070BDF02CEFD3FAE700205B
:1045400070BD00000010014070B586B00024104816
:1045500001940294816941F01001816180690D4EDE
:1045600000F0100004904FF40060022500906946AE
:1045700003953046FDF782FD6802009001AA0120F4
:1045800082E8310069463046FDF778FD06B070BD1F
:10459000001002400010014070B5002400F08AF8BD
:1045A00000F06EF8FFF7A2FF11490870CC2000F070
:1045B0008FF8BE2000F08CF800F052F8054600F0AD
:1045C0004FF8072800D8012405EB002000B23CB1C9
:1045D00004F03EF8BDE870406FF0030104F03FBA0C
:1045E000C04304F035F8BDE87040024904F090B8CB
:1045F0009C000020000080BD10B5FFF7A5FF012240
:1046000091020448FDF743FE00F03AF8BDE810407F
:10461000FFF76CBF0010014070B5104D4FF480647F
:10462000002221462846FDF732FE022002F01CFE41
:10463000012221462846FDF72AFE0C2002F014FE36
:1046400061002846FDF716FE08B1012400E00024B1
:10465000322002F009FE204670BD0000001001402B
:1046600070B500255FF00104FFF7D6FFC001641CA0
:1046700040EA5500E4B2C5B2082CF5D9284670BD11
:1046800070B50B4D4FF48064002221462846FDF79B
:10469000FEFD40F2EE2002F0E7FD01222146284611
:1046A000FDF7F5FDBDE870400F2002F0DDBD000014
:1046B0000010014010B5FFF7E3FFFFF717FFCC2014
:1046C00000F006F8BDE81040442000F001B80000FA
:1046D0002DE9F0410124154F0546A60215F0010F02
:1046E0004FEA55054FF00002314638460BD0FDF732
:1046F000CEFD022002F0B8FD012231463846FDF71A
:10470000C6FD3C200AE0FDF7C2FD3C2002F0ACFDF6
:10471000012231463846FDF7BAFD022002F0A4FD21
:10472000641CE4B2082CD9D9BDE8F0810010014026
:10473000094808B5416941F0010141614069002221
:1047400000F00100009011461020FEF7A1F8BDE82E
:1047500008401020FEF78EB8001002402DE9F04FFF
:1047600085B000244A48009401940294039481691E
:1047700041F010018161816901F0100104918169AA
:1047800041F020018161816901F02001049181697A
:1047900041F004018161816901F0040104918169A2
:1047A00041F0080181618069DFF8E8A000F00800AD
:1047B00041F612060490002231465046FDF767FD8F
:1047C000DFF8D4904FF4F068002241464846FDF7E8
:1047D0005EFDDFF8C8B0002238215846FDF757FDCE
:1047E0004EF24F000325CDE9000569464846FDF726
:1047F00045FCE120CDE9000569465046FDF73EFC49
:104800000096022701260397CDE9016469465046C8
:10481000FDF734FC41F63000CDE900046946484616
:104820000294FDF72BFCCDE90054694658460294EA
:10483000FDF724FC41F20430CDE9000569465846F5
:10484000FDF71CFCCDF800800397CDE901646946B3
:104850004846FDF713FC4FF40140CDE900046946DA
:1048600050460294FDF70AFC0420CDE90004694695
:104870000B480294FDF702FC3820CDE90006CDE993
:10488000024769465846FDF7F9FB05B0BDE8F08FD1
:10489000001002400008014000100140000C0140DF
:1048A000001401400D4810B50B4901600C494160EE
:1048B00000214FF480428160C0E9031241618161AF
:1048C000C1610162FDF76CFE002803D0BDE8104015
:1048D000FDF744B810BD000000540040D001002096
:1048E000A08601000F4810B50D4901604FF4827198
:1048F000416000218160C1604FF400720161C0E934
:104900000512C1610162416281620A21C162FEF742
:10491000CFFA002803D0BDE81040FDF71FB810BD46
:10492000003800402402002010B586B00024194849
:104930000094019402940394049415490594016031
:104940002321C0E9011440F2E731C0E903148021BA
:10495000C0E90541FEF7A4FB08B1FCF7FFFF4FF4E7
:104960008050009069460B48FEF71CFC08B1FCF72C
:10497000F5FF049404A907480594FEF753FB08B11A
:10498000FCF7ECFF0348FEF7D7FB06B010BD0000B4
:10499000002C01407C0200200C4810B50A4901603F
:1049A0004FF4E1314160002181600C22C160C0E917
:1049B00004128161C161FEF701FF002803D0BDE848
:1049C0001040FCF7CBBF10BD00380140C4020020EE
:1049D0000C4810B50A4901604FF41651416000219E
:1049E00081600C22C160C0E904128161C161FEF7DF
:1049F000E5FE002803D0BDE81040FCF7AFBF10BDB6
:104A0000004400400C0300200C4810B50A49016026
:104A10004FF4E1314160002181600C22C160C0E9A6
:104A200004128161C161FEF7C9FE002803D0BDE810
:104A30001040FCF793BF10BD004800405403002015
:104A4000FEE7FEE710B52C4802F00EFCAE2001F0A8
:104A5000D7FD002001F0D4FD102001F0D1FD402051
:104A600001F0CEFDB02001F0CBFD812001F0C8FDAA
:104A7000FF2001F0C5FDA02001F0C2FDA62001F03D
:104A8000BFFDA82001F0BCFD3F2001F0B9FDC02012
:104A900001F0B6FDD32001F0B3FD002001F0B0FD20
:104AA000D52001F0ADFD802001F0AAFDD82001F055
:104AB000A7FD052001F0A4FDD92001F0A1FDF12002
:104AC00001F09EFDDA2001F09BFD122001F098FD1F
:104AD000DB2001F095FD302001F092FD8D2001F0EA
:104AE0008FFD142001F08CFDAF2001F089FDBDE8A1
:104AF000104000F003B8000020A1070070B50024AA
:104B000004F1B000C0B201F07BFD002001F078FD9F
:104B1000102001F075FD0025002001F088FD6D1CBE
:104B2000EDB2802DF8D3641C082CE9DB70BD0000C9
:104B30002DE9FC5FFE4EFF4F06F1120806F11C0145
:104B4000727898F8000049680091FB49002401251B
:104B5000096806F15C0906F1440A06F14C0B0F2ABC
:104B60007ED2DFE812F00F001200A200460112030D
:104B70006004D5042205B005240702085408E4089F
:104B80002E0AAE0AFFF75EFF8CE0FFF7B7FF0023A7
:104B900002221946184601F099FB00230322194608
:104BA000182001F093FB002304221946302001F065
:104BB0008DFB002305221946482001F087FB0023C6
:104BC00006220221184601F081FB00230722022160
:104BD000182001F07BFB002308220221302001F085
:104BE00075FB002309220221482001F06FFB0023FE
:104BF0000A220421184601F069FB00230B2204213C
:104C0000182001F063FB00230C220421302001F066
:104C10005DFB00230D220421482001F057FB0023F7
:104C20000A220621184601F051FB00230B2206211F
:104C3000182001F04BFB002333220621302001F025
:104C400045FB002334220621482001F03FFBB84DEC
:104C50000835287840B910233C220021702000E05C
:104C6000B3E0009401F076FB2878012806D11023E8
:104C70003C2202217020009401F06CFB287802286D
:104C800006D110233C2204217020009401F062FB25
:104C90002878032806D110233C2206217020009496
:104CA00001F058FB7078401C8EE0A14D0835287843
:104CB000697888427BD0E0B910233C220021702023
:104CC000009401F047FB6878012806D110232022C8
:104CD00002217020009401F03DFB6878032806D182
:104CE0001023202206217020009401F033FB287845
:104CF0006870287801281BD110233C2202217020E3
:104D0000009401F027FB687830B91023202200219D
:104D10007020009401F01EFB6878022806D1102351
:104D2000202204217020009401F014FB2878687080
:104D3000287802281CD110233C22042170200094E2
:104D400001F008FB6878012806D1102320220221F7
:104D50007020009401F0FEFA6878032806D1102331
:104D6000202206217020009401F0F4FA287868705F
:104D7000287803281BD110233C22062170200094A0
:104D800001F0E8FA6878022806D1102320220421D5
:104D90007020009401F0DEFA687830B910232022E8
:104DA00000217020009401F0D5FA287868702878E6
:104DB00068B1012811D0022815D0032805D1B07898
:104DC000012802D1B4700C207070BDE8FC9FB0784F
:104DD0000128FAD1B4700320F6E7B0780128F4D1A5
:104DE000B4700420F0E7B0780128EED1B470092047
:104DF000EAE7B046F078514EDFF844914FF4FA7A82
:104E000000287DD0DFF828B10BF11C0BCBF8001087
:104E10000191009803F07AFD4FF07E57B84205DA11
:104E2000DDE9001003F072FDB84219DB019803F0D0
:104E3000D3FB024643A14448FBF72CFA102320225F
:104E400000215020009401F085FA10233E4A0021F1
:104E50003820009401F0ECFADBF80010CBF80410D5
:104E60003168334E24363160706803F081FB1DD009
:104E700036497068884219DA03F018FA02460B4680
:104E800033A1A6F11000FBF705FA1023A6F11002DA
:104E900002213820009401F0CBFA10232E220221A7
:104EA0004820009401F056FA306870602049D9F823
:104EB000000054314E4608600028024600DA524293
:104EC000524501DDC6F800A089464968814216D0E6
:104ED000102321A204214020009401F0A9FA19A175
:104EE00019483268FBF7D6F91023174A04213820F5
:104EF000009401F09DFAD9F80010C9F8041000E000
:104F000035E020211548FDF7B5F903F0B9FB084E4F
:104F100001462C363060706803F02AFB7ED0306882
:104F2000B8427CD1102306210DA2002000941BE082
:104F3000F000002058010020680000206C000020D4
:104F4000AC010020256400002C070020000048422E
:104F5000252E3166000000002020200000100140B6
:104F60002D2D2D2D2D00000001F062FAD1E088F8E2
:104F70000350FFF7C3FD002306221946184601F02F
:104F8000A5F900230E221946102001F09FF90023F5
:104F90000F221946202001F099F910232022002128
:104FA0006020009401F0D6F9FE48006803F014FB7D
:104FB0000246AFF27001FC48FBF76CF91023FA4A85
:104FC00000213820009401F033FA0023102202213E
:104FD000184601F07BF9002311220221102001F074
:104FE00075F9F2483168814201DC084601E0F04879
:104FF000306003F05BF902460B46AFF2AC01ED48BE
:10500000FBF748F91023EB4A02213820009401F005
:105010000FFA00230A220421184601E07BE065E034
:1050200001F054F900230B220421102001F04EF965
:10503000D9F800004946002800DA40425246904222
:1050400002DCD9F8002000E00A60AFF20811D6486F
:10505000FBF720F91023D44A04213820009401F0F2
:10506000E7F92021D448FDF705F901282CD00023C9
:1050700012220621184601F029F9002313220621E5
:10508000102001F023F91023312206212020009462
:1050900001F060F90121C948FDF7ECF801281CD0A6
:1050A000002312220621482001F010F900231322C8
:1050B0000621582001F00AF9102332220621682027
:1050C000009401F047F955E01023AFF26C1206216D
:1050D0000020009401F0ACF9DCE71023AFF280125D
:1050E00006214820009401F0A3F943E00023122296
:1050F0000621184601F0EAF80023132206211020A9
:1051000001F0E4F81023312206212020009401F060
:1051100021F9306870600121A848FDF7ABF803F071
:10512000AFFAA44E014620363060706803F020FAD2
:1051300020D03068B84208D11023AFF2DC1206212B
:105140004820009401F074F912E000231222062195
:10515000482001F0BBF8002313220621582001F05B
:10516000B5F81023322206216820009401F0F2F8ED
:105170003068706098F80210404601297FF425AE2F
:105180008470457088F803401FE6317939B198F88A
:105190000110454688427DD000287CD0D6E035718C
:1051A000FFF7ACFC002316221946184601F08EF8D2
:1051B000002317221946102001F088F80023182236
:1051C0001946202001F082F80023192219463020C8
:1051D00001F07CF87A4D287858B901231A22002171
:1051E000482001F073F801231B220021582001F010
:1051F0006DF8287801280BD101231C2200214820BA
:1052000001F064F801231D220021582001F05EF80E
:10521000287802280BD1012332220021482001F0F6
:1052200055F8012313220021582001F04FF8297866
:1052300088F8001088F80110002316220221184671
:1052400001F044F8002317220221102001F03EF85B
:1052500000231E220221202001F038F800231F2203
:105260000221302001F032F8564DAFF2283151487A
:105270002A68FBF70FF810234E4A022148200094B9
:1052800001F0D6F8102350A202216020009401F012
:10529000CFF801E07AE04DE0464829682830002345
:1052A0000160416016220421184601F00FF8002326
:1052B00017220421102001F009F8202200230421E4
:1052C000104601F003F8002321220421302000F0D1
:1052D000FDFF3E4D2868022805D10023232204212A
:1052E000482000F0F3FF2868012805D1002322227E
:1052F0000421482000F0EAFF2968C9F80010C9F825
:105300000410002324220621502000F0DFFF002398
:1053100025220621602000F0D9FF00232622062145
:10532000184600F0D3FF002327220621102000F0AA
:10533000CDFF2BE001231A220021482000F0C6FFF8
:1053400001231B220021582000F0C0FF28780128EB
:105350000BD101231C220021482000F0B7FF0123BC
:105360001D220021582000F0B1FF287802280BD11F
:10537000012332220021482000F0A8FF012313223C
:105380000021582000F0A2FF28786870B07801282A
:105390007FF4FAAEB470347198F80000444610BB44
:1053A000002315E0680000202C0700200000484280
:1053B0000000C8410401002000100140000C014021
:1053C00059010020780100206D6D00008C01002043
:1053D0001A221946482000F079FF00231B221946A3
:1053E000582000F073FF207801280BD100231C22E5
:1053F0001946482000F06AFF00231D221946582054
:1054000000F064FF207802280BD1002332221946D5
:10541000482000F05BFF002313221946582000F0BB
:1054200055FF0520D0E408BB307900B3FE4FD7E923
:105430000001884215D01023FCA2022150200094C4
:1054400000F0F6FFAFF20451A7F128003A68FAF72E
:1054500021FF1023A7F1280202214820009500F027
:10546000E7FF38687860B078012816D021E0F04F67
:105470003571AFF23051EC483A682838FAF70AFF34
:10548000E94A1023283A02214820009500F0D0FF75
:10549000E548396801604160E5E7B470E24A34717B
:1054A0001023283A02214820009400F0C1FF062072
:1054B000707098F8000001281AD1DB4F1023DBA28E
:1054C0003D607D6002215020009400F0B1FFAFF2FA
:1054D0008C51A7F128003A68FAF7DCFE1023A7F1F7
:1054E000280202214820009400F0A2FF07207070DB
:1054F00098F8000002287FF447AECB481023CDA2D5
:105500000560456002214820009400F091FF44E0CE
:10551000C54831792030006839B1D9F804104D46BA
:10552000884227D0012814D019E035714D46012852
:1055300005D1012322220421482000F0C7FE28685B
:10554000022817D1012323220421482000F0BEFEA7
:1055500010E0012322220421482000F0B7FE286831
:10556000022805D1012323220421482000F0AEFEA9
:1055700028686860B0780128BDD1B4703471D9F85A
:1055800000004C46012805D1002322220421482096
:1055900000F09CFE2068022805D10023232204216C
:1055A000482000F093FE07200EE4B24630799E4E6C
:1055B000323E28B130787178884247D088B128E0EF
:1055C0008AF80450347074700123262206210020CA
:1055D00000F07CFE012327220621102000F076FE39
:1055E00034E0002324220621502000F06FFE002327
:1055F00025220621602000F069FE012326220621D3
:10560000002000F063FE012327220621102000F075
:105610005DFE3078012817D1012324220621502075
:1056200000F054FE012325220621602000F04EFEEA
:10563000002326220621184600F048FE00232722D8
:105640000621102000F042FE307870709AF80210A7
:105650005046012990D13178A1B101298CD18470B3
:10566000047198F800204146022A1CD072493D700E
:105670000A706D496E4A09681160704AD9F80010C5
:1056800011601CE0847004713C70674988F8004028
:1056900088F801400D604D60C9F80050C9F8045009
:1056A0008AF8015070E502223A700C705E4988F861
:1056B00001400D604D60C9F80050C9F80450082140
:1056C0008AF8011060E57079B046E0B3DFF85891D0
:1056D0008A46A9F12009C9F80010009803F016F9CC
:1056E0004FF07E56B04205DC5046009903F00EF9AB
:1056F000B0421ADD504602F0D9FD02460B4650A1D9
:105700005148FAF7C7FD10234F4A02213820009470
:1057100000F08EFE1023202202217020009400F061
:1057200019FED9F80010C9F8041020214748FCF7E9
:10573000A1FD02F0A5FFDFF8F0900146A9F11009E4
:10574000C9F8000000E010E0D9F8040002F010FFF2
:1057500068D0D9F80000B04265D110233CA20421E2
:105760003820009400F064FEC7E088F80550FFF789
:10577000C5F9002316221946184600F0A7FD00239C
:1057800028221946102000F0A1FD002329221946E5
:10579000202000F09BFD10232FA200213020009438
:1057A00000F046FE002306220221184600F08EFD7E
:1057B00000230E220221102000F088FD00230F227A
:1057C0000221202000F082FD2548006802F06EFDD5
:1057D00002460B461AA11C48FAF75CFD10231A4A30
:1057E00002213820009400F023FE0023122204211D
:1057F000184600F06BFD002313220421102000F056
:1058000065FD1023312204212020009400F0A2FD28
:10581000002312220621184600F058FD002313220F
:1058200006211FE06DE05CE02C010020200000005C
:10583000780100202D2D0000590100208C0100204E
:10584000252E3266000000002C07002000100140C9
:105850002D2D2D2D000000002E2E2E2E2E000000AE
:1058600068000020102000F031FD102332220621B4
:105870002020009400F06EFD2021FE48FCF7FAFC89
:1058800001281ED0002314220421382000F01EFD20
:10589000002315220421482000F018FD0121F648BC
:1058A000FCF7E8FC012815D000231422062138203B
:1058B00000F00CFD002315220621482000F006FD13
:1058C00067E01023AFF2780204213820009400F042
:1058D000AFFDE3E71023AFF28802062138200094E1
:1058E00055E0002314220421382000F0EFFC0023AF
:1058F00015220421482000F0E9FCD9F80010C9F86D
:1059000004100121DC48FCF7B5FC02F0B9FEDFF819
:105910006C930146C9F80000D9F8040002F028FE93
:105920001CD0D9F80000B04208D11023AFF2E00239
:1059300006213820009400F07BFD0BE000231422A8
:105940000621382000F0C2FC002315220621482041
:1059500000F0BCFCD9F80010C9F804103878C0B9C0
:1059600000232A221946184600F0B0FC00232B22FF
:105970001946102000F0AAFC00232C2219462020F2
:1059800000F0A4FC1023BEA200213020009400F0FF
:105990004FFD98F80210404601297FF483AEBA49C2
:1059A00084700C703C70457088F805407AE6B079D8
:1059B000D0B35746D7E90001884217D01023B1A2CF
:1059C00002215020009400F033FDAFF68821AB484F
:1059D0003A682038FAF75EFCA84A1023203A0221E0
:1059E0004820009500F024FD38687860B0780128E0
:1059F000DCD1B470B4711023A2A202215020009413
:105A000000F016FDAFF6C4219C48DAF800202038DB
:105A1000FAF740FC994A1023203A022148200094CA
:105A200000F006FD0A20FDE4FFE7B571FFF766F818
:105A300096485F460123C178CAF80010CAF80410DE
:105A40004079CBF80000CBF804000C220021202084
:105A500000F03CFC01230D220021302000F036FC38
:105A600001232D220021402000F030FC01232E22B2
:105A70000021502000F02AFC0021102384A20846B7
:105A8000009500F0D5FC102381A200216020009534
:105A900000F0CEFC00230C220221184600F016FC78
:105AA00000230D220221102000F010FC00232F22E1
:105AB0000221202000F00AFC30220023022110469F
:105AC00000F004FCAFF684317348DAF80020FAF7EE
:105AD000E1FB1023704A02214820009500F0A8FC49
:105AE00010236EA202216020009400F0A1FC00238C
:105AF0000C220421184600F0E9FB00230D220421AA
:105B0000102000F0E3FB002331220421202000F0CC
:105B1000DDFB002311220421302000F0D7FBAFF67B
:105B2000DC315D483A68FAF7B5FB10235A4A042184
:105B30004820009400F07CFC002324220621502001
:105B400000F0C4FB002325220621602000F0BEFBEC
:105B5000002326220621184600F0B8FB0023272246
:105B60000621102000F0B2FB40E74449B07918311B
:105B70000A68D8B3DBF804005F46824217D01023CE
:105B800040A204215020009400F052FCAFF64C419A
:105B90003A483A682038FAF77DFB384A1023203A11
:105BA00004214820009500F043FC38687860B07804
:105BB00001287FF4FBAEB470B471102331A204212C
:105BC0005020009400F034FCAFF688412B48DBF8FD
:105BD00000202038FAF75EFB284A1023203A0421DF
:105BE0004820009400F024FC0B201BE4FFE7B57173
:105BF000AFF6B04121482038FAF74CFB1F4A10237A
:105C0000203A04214820009500F012FCCFE71B4FFA
:105C1000B079283F28B13878797888425DD080B152
:105C200027E0B5713C707C700123262206210020FC
:105C300000F04CFB012327220621102000F046FB38
:105C40004BE0002324220621502000F03FFB0023DC
:105C500025220621602000F039FB0123262206219F
:105C6000002000F033FB012327220621102000F042
:105C70002DFB15E000100140000C01402401002024
:105C800021202020200000005A0100207D0000205B
:105C900020202020000000002C0700206D73000051
:105CA0003878012817D1012324220621502000F042
:105CB0000DFB012325220621602000F007FB0023B5
:105CC00026220621184600F001FB00232722062188
:105CD000102000F0FBFA38787870B07801287FF453
:105CE00065AE3878A8B10128F9D1B470FA48B4711A
:105CF0009AF80010C1709BF8001041710122022136
:105D0000F648FCF7C4FA0722F349F548FDF74EFEC2
:105D1000BEE2F149B470B471CA78CAF80020CAF87A
:105D200004204979CBF80010CBF80410B0E2B07928
:105D300030B1EC4F3878797888427DD0E8B3DBE039
:105D4000B571FEF7DBFE0622E749E84800F086FC65
:105D5000E5490020E44E0C3936F8102021F81020D7
:105D6000401CC0B20628F7D300230A221946184661
:105D700000F0ACFA00230B221946102000F0A6FA1E
:105D8000D84F387830B91023D9A200214820009587
:105D900000F04EFB3878012806D11023D6A200214E
:105DA0004820009500F044FB3878022808D11023E1
:105DB0000021D3A24820009500E096E000F038FBD7
:105DC000002335220221184600F080FA00233622F3
:105DD0000221102000F07AFA00232922022120203B
:105DE00000F074FA00231A220221302000F06EFA2B
:105DF000387870B93288AFF6B461BB481C38FAF70E
:105E000049FAB94A10231C3A02214820009400F0B4
:105E10000FFB387801280ED17288AFF6D861B248EE
:105E20001C38FAF737FAB04A10231C3A02214820EE
:105E3000009400F0FDFA00E074E0387802280ED1FA
:105E4000B288AFF60071A8481C38FAF723FAA64AC0
:105E500010231C3A02214820009400F0E9FA0023A4
:105E60002D220421184600F031FA00232E220421AD
:105E7000102000F02BFA002329220421202000F01A
:105E800025FA00231A220421302000F01FFA9E4830
:105E9000006802F0BDFB82B2AFF6587192481C3820
:105EA000FAF7F8F9904A10231C3A0421482000948C
:105EB00000F0BEFA002324220621502000F006FA4A
:105EC000002325220621602000F000FA002326226C
:105ED0000621184600F0FAF902B00023BDE8F05F91
:105EE00027220621102000F0F1B9102380A2002102
:105EF0004820009500F09CFA3878012806D110233C
:105F00007DA200214820009500F092FA38780228FE
:105F100006D110237AA200214820009500F088FACB
:105F200038787870B07801287FF440ADB470B471DF
:105F30003878A0B910236EA200214820009400F008
:105F400077FA694871A102881C38FAF7A3F9664A02
:105F500010231C3A02214820009400F069FA387896
:105F6000012814D1102364A200214820009400F0DD
:105F70005FFA5D4865A142881C38FAF78BF95A4AE6
:105F800010231C3A02214820009400F051FA38787E
:105F9000022814D110235EA200214820009400F0B2
:105FA00047FA514859A182881C38FAF773F94E4ACA
:105FB00010231C3A02214820009400F039FA0D20E9
:105FC00031E5B07988B3DFF81C818A4608F10E0804
:105FD000C8F80010009802F099FC4FF07E5948452F
:105FE00005DC5046009902F091FC484514DD50460E
:105FF00002F00EFB82B23C4844A11C38FAF74AF981
:10600000394A10231C3A04214820009500F010FA68
:10601000D8F80010C8F80410F179E1B10F203E4A19
:1060200001291CD0022944D021E0FFE72D48B57199
:106030000E30006802F0ECFA82B22B4833A11C3813
:10604000FAF728F9284A10231C3A04214820009521
:1060500000F0EEF90BE031483C70056005E0304996
:10606000146008602D48056029E02E480470B0785F
:1060700001287FF49BAC2A48B470B47105602948AC
:106080003C7004702548056016480E30006802F028
:10609000BFFA82B214481DA11C38FAF7FBF8124A65
:1060A00010231C3A04214820009400F0C1F90E206E
:1060B000B9E41B49146008601849022008603D706B
:1060C000D3E7084FB179BF1C387821B1797888427D
:1060D00060D048B377E028E07D0000200008014050
:1060E0000C030020FE0000204807002000F00108FB
:1060F000233235200000000023353020000000004E
:1061000023313130000000006800002025640000C9
:1061100023313130200000006C0100208C01002070
:10612000780100205901002035E0B571B8B900238D
:1061300024220621502000F0C9F800232522062140
:10614000602000F0C3F8012326220621002000F081
:10615000BDF8012327220621102000F0B7F8387877
:1061600001284DD1012324220621502000F0AEF851
:10617000012325220621602000F0A8F80023262212
:106180000621184600F0A2F800232722062110203D
:1061900000F09CF834E0002324220621502000F077
:1061A00095F8002325220621602000F08FF80123B6
:1061B00026220621002000F089F80123272206214B
:1061C000102000F083F83878012817D10123242209
:1061D0000621502000F07AF80123252206216020B4
:1061E00000F074F8002326220621184600F06EF80D
:1061F000002327220621102000F068F838787870F4
:10620000B07801287FF44EAA3878012836D1DFF81B
:106210008880B470B47198F8000020B101280AD0C9
:10622000022810D016E01C480E30006802F0F0F989
:106230001A4908800EE018480E30006802F0E8F9AC
:106240001649488006E014480E30006802F0E0F974
:106250001249888006221149114800F00DFA0F48B2
:1062600010490C30008808603C707C7088F8004051
:1062700088F801407570B0780128C3D138780028BB
:10628000C0D1B470B47104483C707C700470447028
:106290007570BDE8FC9F0000FE0000203C07002058
:1062A00000F001085401002010B50446B031C8B216
:1062B00000F0A6F9102040EA141000F0A1F904F053
:1062C0000F00BDE8104000F09BB900002DE9F0413F
:1062D00007461F484D1C00EB4216FBB1012B1BD19A
:1062E0003846FFF7E1FF0024305DC043C0B200F044
:1062F0009EF9641CE4B2102CF6D3E9B23846FFF7DD
:10630000D3FF00243019007CC043C0B200F08FF9E5
:10631000641CE4B2102CF5D3BDE8F0813846FFF7D9
:10632000C3FF0024305D00F082F9641CE4B2102C3D
:10633000F8D3E9B23846FFF7B7FF00243019007CE4
:1063400000F075F9641CE4B2102CF7D3E4E7000008
:106350001C9300082DE9F0418046203A002406985D
:106360000E46D7B2B8F17F0F02D9B61CA046F6B2DE
:10637000102B11D031464046FFF796FF2A4907EB14
:10638000470001EB4005285D00F051F9641CE4B2C0
:10639000062CF8D3BDE8F081244D20B30128F9D1B3
:1063A00031464046FFF780FF04EB0710285CC043EE
:1063B000C0B200F03CF9641CE4B2082CF4D3761CA3
:1063C000F1B24046FFF770FF5FF0000404EB0710E6
:1063D0002844007AC043C0B200F029F9641CE4B23A
:1063E000082CF3D3D6E731464046FFF75DFF00BFE8
:1063F00004EB0710285C00F01AF9641CE4B2082CC6
:10640000F6D3761CF1B24046FFF74EFF5FF0000472
:1064100004EB07102844007A00F009F9641CE4B288
:10642000082CF5D3B6E70000048B00082C8D00087B
:106430002DE9F843994617460E4604460025DDF837
:1064400020800FE04B4631462046CDF80080FFF714
:1064500081FF0834E4B2782C02D90024B61CF6B2CD
:106460006D1CEDB27A5D002AECD1BDE8F8832DE910
:10647000F041164605460C460F461AE0761EB44219
:1064800008DA55F8271055F8260002F00DFA01D861
:10649000F4E7641CB44206DA55F8271055F82400D6
:1064A00002F002F9F5D905EB860105EB840000F056
:1064B0006AF9B442E3DB05EB840105EB870000F0E9
:1064C00062F92046BDE8F08170472DE9F04114469D
:1064D0000D460646A1420BDAFFF7C9FF0746421EEA
:1064E00029463046FFF7F1FF2246791C3046EEE799
:1064F000BDE8F08141780A02817811430A02C1782F
:106500000079114340EA01207047000070B5114E38
:10651000002210213046FBF7BAFE0A2000F09EFE52
:10652000102000F0DDFC00F017F8044600F014F82D
:10653000054600F011F8014645EA042041EA00242E
:106540000A2000F08BFE012210213046FBF79FFE4F
:10655000204670BD0008014070B5134E0022202176
:106560003046FBF794FE0024012220213046FBF741
:106570008EFE012000F072FE6806050E40213046B6
:10658000FBF778FE08B145F00105002220213046D6
:10659000FBF77DFE012000F061FE641CE4B2082CD4
:1065A000E2D3284670BD00000008014070B50C4DD4
:1065B000002210212846FBF76AFE232000F090FC01
:1065C0005FF00004FFF7C8FF641CE4B2042CF9D3A9
:1065D0002846BDE8704001221021FBF758BE00009C
:1065E000000801400148FCF7F3BB00002402002032
:1065F00010B5406A0021C187C186FCF7E7FB10BDDA
:1066000010B5044600F080FF782000F04FFF00F046
:10661000FFFE002000F04AFF00F0FAFE204600F0E6
:1066200045FF00F0F5FEBDE8104000F08DBF10B54D
:10663000044600F069FF782000F038FF00F0E8FE23
:10664000402000F033FF00F0E3FE204600F02EFF74
:1066500000F0DEFEBDE8104000F076BF10B500236C
:1066600006E000BF30F8024B21F813405B1C9BB2E0
:106670009342F7D310BD00002DE9F05FA0F1006454
:1066800015468A468346B4F5802F5FD2FBF7E2FCBD
:10669000E70AC4F34906C6F58064A54200D82C4633
:1066A000DFF8AC904FF0006000EBC72080464FF45D
:1066B00080622749FFF7D2FF00204FF6FF7106E006
:1066C000331839F813208A4203D1401C80B2A0420B
:1066D000F6D3A0422ED24046FBF7B8F94CF2503028
:1066E000FBF78AF91B48016921F0020101610020D2
:1066F000494606E03AF810208319401C21F813207F
:1067000080B2A042F6D3124940464FF4806200BFE7
:1067100000F022F8A54215D0281B0AEB440A0BEB27
:10672000440B002685B24FF480647F1CA542B9D883
:106730002C46B7E74CF25030FBF75EF92246514643
:106740005846E5E7BDE8F05FFBF73ABCBDE8F09FCF
:10675000C0070020002002402DE9F04116460F46F8
:10676000054600240AE000BF37F81420002329461C
:106770000120FBF72FFC641CA4B2AD1CB442F3D380
:10678000BDE8F081704702680B6803600A607047DB
:106790004FF0E0210428086903D020F004000861CC
:1067A000704740F00400FAE7FCF70CB830B58FB042
:1067B00028216846F9F745FE14210AA8F9F741FE99
:1067C00001210804CDE9001000240294022504915F
:1067D000CDE907504FF4E01009906846FCF766F9E0
:1067E00060B90F20CDE90A058020CDE90C04022113
:1067F0000AA80E94FCF77EF8002801D0FBF7AEF84B
:106800000FB030BD704700000148FCF73ABD0000F2
:106810007C020020F0B502681C4B1D4D1D4E1E4F22
:106820001E4C4FF0804C984209D0A04207D06045E2
:1068300005D0A84203D0B04201D0B84204D122F022
:10684000700E4A6842EA0E02984209D0A04207D070
:10685000604505D0A84203D0B04201D0B84203D170
:1068600022F44075CA682A434D6922F080022A4307
:1068700002608A68C2620A688262984201D0A042BD
:1068800001D10969016301214161F0BD002C014082
:106890000004004000080040000C004000340140AB
:1068A00010B5846842EA032224F47F440A43224359
:1068B000826010BD826822F070020A4342F0070134
:1068C0008160704710B5036A046A24F00104046211
:1068D000846924F0F00444EA021423F00A020A4313
:1068E0008461026210BD10B5036A046A24F01004CA
:1068F0000462846923F0A00324F4704444EA023261
:1069000043EA01118261016210BD000070B586B0DA
:10691000104800240294816941F008018161806976
:106920000D4E00F0080004904FF42040009001202C
:1069300002250190694603953046FBF79FFB6803EB
:10694000CDE90004694603953046FBF797FB06B096
:1069500070BD000000100240000C014070B50546FB
:106960000C4600220C4811468154521CD2B2052A12
:10697000FAD300221146284600F010F800221146F2
:10698000284600F00BF804483038016B216090F87D
:106990003400207170BD0000D00000202DE9F05FB0
:1069A0000546174600200E46444A04460146115447
:1069B000401CC0B20528FAD3002280214048FBF7D2
:1069C00066FC642000F030FC17B145F0800501E062
:1069D00005F07F05DFF8EC904FF4005A0122514694
:1069E0004846FBF754FC00274FF4804B0022D0466A
:1069F00051464846FBF74BFC280601D5012200E032
:106A000000224FF400414846FBF741FC6806050EA2
:106A10000122C24641464846FBF739FC142000F0EB
:106A200003FCDFF89880484698F80010490088F881
:106A300000105946FBF71EFC28B198F8001041F0F1
:106A4000010188F800107F1CFFB2082FCED3002769
:106A5000C8460022D14651464046FBF718FC002E9E
:106A600001DA012200E000224FF400414046FBF72A
:106A70000EFC7600012249464046FBF708FC142034
:106A800000F0D2FB640059464046FBF7F3FB08B127
:106A900044F001047F1CFFB2202FDAD30748210EF7
:106AA000012205704170210C8170210AC1700471AE
:106AB000BDE8F05F80210248FBF7E9BBD000002071
:106AC00000100140000C014001B501226946024856
:106AD000FCF76CFF08BD0000C402002010B5406A3E
:106AE0000021C185C184FCF732FD10BD70B5446A38
:106AF0002068406994F84110C0F3C0100025212996
:106B000004D118B1E584204600F08EF82068406971
:106B100094F84210C0F38010222904D118B1E58501
:106B2000204600F05AF8606C40F010006064204687
:106B3000FCF70DFD70BD10B50146406A0968096893
:106B40004FF0000289062ED4C28501680C3151E84D
:106B5000003F23F4807341E80034002CF5D1016834
:106B6000143151E8003F23F0010341E80034002CC8
:106B7000F5D10168143151E8003F23F0400341E8AA
:106B80000034002CF5D1202180F84210016B01293E
:106B900009D101680C3151E8003F23F0100341E8AE
:106BA0000034002CF5D14263016B012902D0FCF7BF
:106BB000FBFE10BD818DFCF7C9FC10BD10B5406A0D
:106BC00001214163016B012902D0FCF7EEFE10BDEB
:106BD000818D4908FCF7BAFC10BD01680C3151E801
:106BE000002F22F4907241E80023002BF5D10168B8
:106BF000143151E8002F22F0010241E80023002B5C
:106C0000F5D1016B012909D101680C3151E8002F40
:106C100022F0100241E80023002BF5D1202180F85A
:106C2000421000210163704701680C3151E8002FC8
:106C300022F0C00241E80023002BF5D1202180F88A
:106C40004110704708B590F84210222901D0022067
:106C500008BD82684FF480539A4201D1016921B185
:106C6000816A9A421BD04AB10AE00268816A52687E
:106C7000C2F308020A80816A891C08E0026972B1C5
:106C80000268526802F07F020A70816A491C8162C0
:106C9000C18D491E0904090CC18503D01BE002689F
:106CA0005268F1E70168CA6822F02002CA600168F0
:106CB000CA6822F48072CA6001684A6922F001023F
:106CC0004A61202180F8421000214163026B012AB1
:106CD00003D0FCF769FE002008BD016301680C3198
:106CE00051E8002F22F0100241E80023002BF5D1DB
:106CF00001680A68D20602D50A6849680091818D48
:106D0000FCF724FCE7E7000070B504460068016961
:106D1000E26821F44051114301612169A0680843F0
:106D2000616908432168CA6841F20C639A430243CF
:106D3000CA6020684169A26921F440711143416130
:106D40001E492068884202D1FBF77AFE01E0FBF77A
:106D500067FE00EBC00101EB001260686421800057
:106D6000B2FBF0F3B3FBF1F36FF018067343B2FB21
:106D7000F0F5B2FBF0F605EB8305322303EB0515C6
:106D8000B5FBF1F5B6FBF1F605F0F00505EB0615E0
:106D9000B2FBF0F6B2FBF0F0B0FBF1F06FF01802CE
:106DA000504306EB800003EB0010B0FBF1F02168CC
:106DB00000F00F002844886070BD000000380140DA
:106DC00038B5816204468285002013466064222221
:106DD00084F84220E56B1B4AAA62E56B1A4AEA6214
:106DE000E56B1A4A2A63E26B50630A462168E06B3E
:106DF000091DFBF7ADF82068016840680090206924
:106E000048B120680C3050E8001F41F4807140E820
:106E10000012002AF5D12068143050E8001F41F01C
:106E2000010140E80012002AF5D12068143050E832
:106E3000001F41F0400140E80012002AF5D1002077
:106E400038BD0000376B0008BD6B0008ED6A000814
:106E500010B50948FCF77CFB08480068800609D596
:106E60000648001D00680649C0B20870BDE8104021
:106E700000F05ABF10BD0000C402002000380140DD
:106E80000000002010B50548FCF762FBBDE810408B
:106E9000062203490148FCF732BB00000C03002026
:106EA0004C0000200148FCF753BB000054030020B5
:106EB000002104E00222521C7D2AFCD3491C81429D
:106EC000F8D37047FEE710B503464078002203E090
:106ED0009C5C6040521CD2B28A42F9D310BD0000C3
:106EE00070B5134E05460024280601D5012200E0A6
:106EF000002280213046FBF7CAF96806050E0A20F9
:106F000000F0B2F9012220213046FBF7C0F90A2037
:106F100000F0AAF9002220213046FBF7B8F90A2038
:106F200000F0A2F9641CE4B2082CDDD370BD0000AF
:106F3000000801402DE9F041124F15460E46044667
:106F4000002210213846FBF7A2F90C20711E00EA3E
:106F5000840001F00301084340F04000FFF7C0FF48
:106F6000002405E02878FFF7BBFF641CE4B26D1C29
:106F7000B442F7D33846BDE8F04101221021FBF7B7
:106F800086B90000000801402DE9F0410E4619497C
:106F90000546487800282AD00020884648601649CF
:106FA00001F5C87451F8202044F82020401CC0B2DC
:106FB0006428F7D3632200211048FFF786FA681E81
:106FC000C7B2D8F8040005E054F8271001F09AF988
:106FD0007F1CFFB2B742F7D30746701B4446401CE4
:106FE00001F036FB0146384601F000FA6060BDE86A
:106FF000F0810000900000200C0400209C0500207F
:107000000F4810B501680F4C012912D10021016011
:107010002078642801D2012100E000214143217041
:107020000420FAF725FD084A217842F82100491C7E
:1070300021702078642801D10120607010BD00000B
:1070400008000020900000200C040020490050EAB5
:10705000C12018BF04204A0D18BF40F0010040F2C3
:10706000FF72B2EB515F08BF40F00200012808BF79
:10707000052070470907090E002804DB00F1E02015
:1070800080F80014704700F00F0000F1E02080F855
:10709000141D704730380A2801D2012070470020A3
:1070A000704700002DE9F047524C207850B9062275
:1070B00051495248FFF7D2FA4F48514900880860B9
:1070C0000120207000F058FA4E480027016831B3C3
:1070D0004849076014311220FFF740FC454814303E
:1070E000FFF708FA206148496F20FFF737FC464850
:1070F000FFF700FA45490860C0F30900608000F01E
:1071000005F900F0CBF8FDF747FAA060FDF710FD98
:107110004B211920FFF738FF606000F0F3FDFFF707
:107120006FFF3B493B4800F0A5FBFAF731FAFAF74D
:107130001DFB394E394D4FF4805930784FF4006AB9
:1071400048B9012249462846FBF7A1F801225146D9
:107150002846FBF79CF83078012820D1DFF8C08062
:10716000D8F8000001280CD1002249462846FBF738
:107170008EF8012251462846FBF789F8307801281D
:107180000DD1D8F80000022831D101224946284605
:10719000FBF77DF8002251462846FBF778F8307857
:1071A000022801D0032822D1E06864280AD10022F5
:1071B00049462846E760FBF76AF800225146284610
:1071C000FBF765F817480168002910D00760E068F0
:1071D000401CE06002280AD149462846E760FBF7D8
:1071E0004EF851462846BDE8F047FBF748B8BDE8E1
:1071F000F0870000640000204807002000F001082C
:107200005401002030000020E8000020E4000020AD
:107210000080ED440000C8425801002000080140F1
:107220008C0100201000002000E000BF401EFCD2B6
:107230007047000010B56FF00400FFF7A9FA04488A
:1072400004490068B0FBF1F00349087010BD00006C
:107250006000002000127A0088000020002100E079
:10726000491C8142FCDB70470B49097848434FF0C9
:10727000E021486100228A61086940F0010008614C
:107280000869C30701D0C003FAD5086920F00100DE
:1072900008618A61704700008800002070B51548B9
:1072A000154C164D0279C179C2EB02621144427944
:1072B0008079C2EB0242C0EB002010440844104E1B
:1072C000E064010206D5C043206500F0DAFE2A46DC
:1072D0000C4B04E0206500F0D4FE2A460A4B00F077
:1072E000E7FE0022334600F0E3FE00F09BFE6065FF
:1072F00070BD0000900700205801002050000028B9
:1073000000408F40000094BE0000943E70B5384CA1
:10731000384D3949207868706078A870E078421C50
:107320000B5C052B07D0052801D2012000E00020CE
:107330005043E07032E0052A01D9012200E000222A
:10734000A2EB820200EB42020A4452782A71821CAC
:10735000052A01D9012200E00022A2EB820200EB03
:1073600042020A4492786A71C21C052A01D901229C
:1073700000E00022A2EB820200EB42020A44D27833
:10738000AA71021D052A01D9012200E00022A2EB08
:10739000820200EB420008440079E871174921207D
:1073A000FFF7DCFA1548FFF7A5F8154908601549FD
:1073B0000968401A642148434FF4205190FBF1F0D2
:1073C000A080010A2972687220210F48FAF752FF43
:1073D00048B101210D48FAF74DFF30B194F834005F
:1073E000801CE87070BD0120FBE70220F9E7000077
:1073F00058010020900700204C000020D5000020FC
:10740000C40000208400002000100140000C014056
:1074100010B50E4C002280212046FAF738FF00F00C
:107420003FF8012240212046FAF731FF00F038F8FA
:10743000002240212046FAF72AFF00F031F82046CA
:107440000122BDE810408021FAF721BF000C014065
:1074500000B585B0002002900F48816941F0080115
:107460008161816901F008010491816941F008019D
:1074700081618069694600F008000490C020009096
:1074800011200190032003900448FAF7F7FD00F063
:107490005BF805B000BD000000100240000C014088
:1074A0000020401CC0B20A28FBD3704770B5154EAF
:1074B00005460024280601D5012200E00022802193
:1074C0003046FAF7E4FEFFF7EBFF01224021304699
:1074D000FAF7DDFEFFF7E4FF002240213046FAF71D
:1074E000D6FE072C04D1012280213046FAF7CFFEC8
:1074F0006806050EFFF7D4FF641CE4B2082CD9D34C
:1075000070BD0000000C014010B50E4C012280211E
:107510002046FAF7BCFE012240212046FAF7B7FECA
:10752000FFF7BEFF002280212046FAF7B0FEFFF7EA
:10753000B7FF002240212046FAF7A9FEBDE810401F
:10754000FFF7AEBF000C014010B50A4C00228021AD
:107550002046FAF79CFE012240212046FAF797FECA
:10756000FFF79EFF20460122BDE810408021FAF778
:107570008EBE0000000C01402DE9F04F8E4B01271C
:1075800002261878012802D18C4807701E708C489A
:107590005D788D4C02788B488C49DFF834E2DFF857
:1075A0003492DFF834A2921E4FF0000C012D7BD1F3
:1075B00025460D2A2D780DD2DFE802F0078810222B
:1075C0002B3C8843505D657E97000578032D02D2E1
:1075D0006D1C05707AE080F800C077E0A5F1010825
:1075E000002D01D04FF0010508FB05F802D14FF046
:1075F000010501E04FF0000508EB4505257065E049
:107600005DBB0D68012D01D96D1E00E00F250D60D9
:107610005CE0DEF80050022D09D04FF00008012D8B
:1076200000D0002508EB4508CEF800804EE04FF072
:107630000108F6E7DFF8A4B11FE000BF8BF8008077
:1076400044E0D9F80080B8F1050F02D9A8F101088B
:1076500001E04FF00A08C9F8008037E0DAF800804E
:10766000B8F10A0F02D9A8F1010801E04FF014089F
:10767000CAF800802AE0DFF868B19BF80050BDB37B
:107680004FF00008DAE7DFF85CB19BF80050A5F195
:107690000108002D02D000BF4FF0010508FB05F8DE
:1076A00003D14FF0010502E011E04FF0000508EBB7
:1076B00045058BF8005009E04B4D95F80080B8F176
:1076C000000F02D085F800C000E02E705E709D783B
:1076D000012D6BD10D2A68D2DFE802F00E6715206C
:1076E0002A39673B454F54606A00DFF800B1C4E7B0
:1076F000FFE74FF00108A1E7017809B1491E00E05A
:107700000321017051E020780146401C022901D27A
:10771000012100E000214843207046E0207808BBAA
:1077200008680F2802D2401C08603EE00F603CE071
:10773000DEF80010022908D00022012900D0002123
:1077400002EB4101CEF800102FE00122F7E72348B9
:1077500014E0D9F800100A2901D2491C00E00521E3
:10776000C9F8001021E0DAF80010142901D2491CF0
:1077700000E00A21CAF8001017E019480178C9B1E1
:107780000021BEE7174908780246401C022A01D2B0
:10779000012200E000225043087006E01248017800
:1077A00011B180F800C000E007709E70BDE8F08F56
:1077B0000E48E3E70121A4E78A000020F200002040
:1077C000F1000020F8000020020100202C01002020
:1077D0004C010020340100203C010020FA00002070
:1077E000FC000020FE000020F70000200001002027
:1077F000FAF7F0FFFEF7DAFFFCF7B0FFFCF798FFAF
:10780000FDF792F8FDF74EF8FDF76CF8FDF7C4F8B8
:10781000FDF7DEF8FDF7F8F8FFF70CFDFFF718FEAF
:10782000FDF710F9114C012211032046FAF72FFD44
:107830000122D1022046FAF72AFD0D48FFF714FD78
:10784000002202212046FAF722FDFCF77DFEFCF71C
:10785000D3FEF9F7F9FDFFF759F800F0CDFAFCF780
:10786000E9FD00BFFFF71EFCFCE700000008014037
:1078700080841E002DE9F0410D4D884600260D4FF5
:107880000D4C296801F010F805D82068012802D0B5
:107890003E70012020604146286801F005F805D8B7
:1078A0002068022802D03E7002202060BDE8F081EE
:1078B00068000020580100208C0100202DE9F05FB5
:1078C000C74EDFF820A33146B278896BC648DFF88F
:1078D0001C930227C64D0024491C4FF0010B42F2B5
:1078E0001078082A7ED2DFE802F0A9040B87B0CC1A
:1078F000FEFDC04874628470B463B4622C705CE1B5
:10790000B06800F0A5FEBC4F396800F0CDFE48D845
:107910000021084600F0F4FA47460AE00021084634
:1079200000F0EEFA306C401C3064B84228DC287855
:1079300030B328780128F1D0B0492120FFF70EF8A4
:10794000AE48FEF7D7FDAE490860AE4970640978CD
:10795000192917D0322918D06E291AD0D2291BD054
:10796000B464A9480168D1B10460B06B401CB06335
:10797000F169884262D3B078401CB070B46374E09F
:107980003464D9E700F59B2001E000F50C20B064D9
:10799000E7E700F59110FAE700F50710F7E7B06B9D
:1079A000E6E7F06A08B9C6F82CB0B068963800F07F
:1079B0004FFE396800F078FFD9F800004C4601D836
:1079C000924901E043F6982188420ED001222720F7
:1079D0002160FEF7E3FF2068012241082520CAF854
:1079E000001000E02AE0FEF7D9FF96F8340088493D
:1079F00000F086FA062020E0D9F8000047F2305166
:107A00004C4688420CD0012227202160FEF7C6FF99
:107A10002068012241082520CAF80010FEF7BEFFA9
:107A2000706968B15FEA802196F8340000F068FA66
:107A30002878002802D1B078401CB070BDE8F09FD3
:107A4000306A00EB8000C102EEE7724802680AB1BA
:107A50000460B163B1693220B1FBF0F0B16B8842D0
:107A6000ECD80520B463B070F462FFF74FFC6A48AD
:107A7000604B0A220188BDE8F05F4FF2010000F080
:107A800069B92021FAF7F6FB28B9706B012802D0FA
:107A9000C6F834B008E001216048FAF7EBFB30B9D2
:107AA000706B022803D07763B4703470C6E703208C
:107AB000B07052492120FEF751FF5048FEF71AFDE1
:107AC000DFF83C914FF0070AC9F80000B16CF1B142
:107AD000884241D3706B02283ED00021084600F056
:107AE0000FFA0EE06BE057E00021084600F008FABC
:107AF000306C401C3064404501DD346426E0287859
:107B000018B128780128EFD020E0346420E0F06834
:107B100000F09EFD3849096800F0C6FD1CD8706B66
:107B2000022819D00021084600F0EAF90BE00021F4
:107B3000084600F0E5F9306C401C30644045DCDC60
:107B400028780028E1D028780128F0D0287818B9C2
:107B5000C6E90D7486F802A0D9F80000716C88425D
:107B6000A4D8706B0228A1D10021084600F0C8F902
:107B70000AE00021084600F0C3F9306C401C306474
:107B8000404507DC287828B128780128F1D03770E3
:107B9000B47053E73464FAE72021FAF76BFB18B9A5
:107BA000706B01287FF474AF01211C48FAF762FB67
:107BB00018B9706B02287FF476AFB7703EE71848AB
:107BC00002680AB10460B163B06B6421B0FBF1F0EC
:107BD000F1698842DDD30320B070B4632EE7000062
:107BE00058010020AC00002000100140B00000202F
:107BF000A00000209007002068000020D500002091
:107C0000C4000020B501002040000020C0D40100C5
:107C10000070170028000020B8010020000C01406F
:107C20002000002070B520212A48FAF723FB2A4CB7
:107C3000002528B9606B012802D00120606346E06E
:107C400001212648FAF716FB022120B9606B0228B1
:107C500001D061633BE0A078062807D2DFE800F09E
:107C60000603071B1D37A563A562A17070BD60697F
:107C700060B1810294F8340000F042F918480078AD
:107C80000028F3D1A078401CA07070BD206A00EBE2
:107C90008000C102EEE70420F6E712480168A1B1B6
:107CA0000560A06B401CA0630A28EED30520A563E5
:107CB000A070FFF72BFB0D480B4B0A220188BDE893
:107CC00070404FF2010000F045B8A06BECE7A570E2
:107CD000257070BD0010014058010020000C0140CB
:107CE000A00000202800002090070020B8010020FC
:107CF0000348002141708170C170FCF79BBB0000FC
:107D0000B001002007484178012902D18178491C3F
:107D10008170C178002904D08078884201D3FFF7B0
:107D2000E7BF7047B00100200346094800B500785E
:107D30003C2807D20A2000F053F818465DF804EBFF
:107D4000F9F7B2BDFFF7D4FF5DF804EBFCF772BBA7
:107D5000B001002070B590B0052514468DF8005094
:107D600004F10B052E0A8DF801608DF802500D0A02
:107D70008DF8041019498DF803500022C9888DF838
:107D800008000D0A8DF805508DF80610010A8DF8CF
:107D900007106D4604E0985CA918521C4872D2B2D4
:107DA000A242F8D304F10900C1B22846FFF78BF8CC
:107DB000291900264872002088721B20C8720C34D2
:107DC00007E0A85DFEF780FE3220FFF771F8761C11
:107DD000F6B2A642F5D310B070BD0000B00100208D
:107DE000002805D0034901224A7000228A70C87019
:107DF00070470000B001002010B5012204210020CE
:107E0000FEF7CCFD012239490A20FEF7C7FD012209
:107E100037491020FEF7C2FD01220A211120FEF78A
:107E2000BDFD012200211320FEF7B8FD0122002133
:107E30001420FEF7B3FD012200211520FEF7AEFD50
:107E40002C4C012220206168FEF7A8FD01220021B0
:107E50002120FEF7A3FD012200212320FEF79EFD35
:107E6000012224206169FEF799FD01222620A169E3
:107E7000FEF794FD01222520E168FEF78FFD012227
:107E800027202169FEF78AFD01222A20E169FEF7F9
:107E900085FD01222820216AFEF780FD01221021A4
:107EA0002B20FEF77BFD012243F6FF712C20FEF70D
:107EB00075FD01222D20A168FEF770FD0122002131
:107EC0003420FEF76BFD01220B496C20FEF766FDA6
:107ED00001224FF440016D20FEF760FD0122BDE854
:107EE000104006497020FEF759BD0000000408004C
:107EF000020A0700A0000020C30001001E000CC4FD
:107F00002DE9F04101263B4C0F46002548B12146A2
:107F10004FF47A78097801282AD0022826D1E1B3D3
:107F20003CE0344922203A31FEF718FD31483A301E
:107F3000FEF7E0FA2F49A06235312120FEF70EFD51
:107F40002C483530FEF7D6FA6062A06A68B1267018
:107F50002946012220206560FEF720FD616ABDE808
:107F6000F04101222D20FEF719BD2570BDE8F081FA
:107F7000A1B92049267035312120FEF7EFFC1D48BC
:107F80003530FEF7B7FA656060622946012220208D
:107F9000FEF704FD606AC11923E00FE02078012894
:107FA000E4D1144935203F31FEF7D8FC11483F3069
:107FB000FEF7A0FAE0628005D7D4D7E70D49267016
:107FC00035312120FEF7CAFC0A483530FEF792FA17
:107FD00065606062294601222020FEF7DFFC606AAE
:107FE000C11B01222D20FEF7D9FC4046FFF71CF9EA
:107FF000D4E70000A000002010B500290AD00878BE
:10800000002807D005487844F8F7FAFD002801D089
:10801000002010BD0248784410BD0000CA1A0000BC
:10802000C21A00004FEA41034FEA5353A3F580639D
:10803000D3F11E03C8BFD3F1210C0CDD4FF0004279
:1080400042EAC12242EA505232FA03FC8CEAE17C55
:10805000ACEBE1707047102BC4BF0020704703F5F4
:10806000787CBCF1FF3F04D06FF0004282EA21002F
:10807000704770B500F0C6F8499224800020704720
:10808000F2E710F0004248BF4042B0FA80F310FA25
:1080900003F10AD0C3F11D0303F580634FEA415099
:1080A00002EB035202EBD12170474FF00000704702
:1080B000DFF848C170B51CEA111E1EBF1CEA13157B
:1080C0009EEA0C0F95EA0C0F00F06F8081EA030422
:1080D00023EA4C134EEAD47E21EA4C1141F480117C
:1080E00043F48013AE44A1FB024CA0FB0365AEF148
:1080F0007F7E361955EB0C05A1FB034C4CF10003B8
:10810000A0FB021C16EB0C06654153F1000309426B
:1081100018BF46F0010613F4007F0BD14FEA03317C
:108120004FEA0530340341EA155140EA16506FF02A
:1081300003020AE04FEAC3214FEAC520F40241EAF4
:10814000555140EA56506FF0020202EB2E4201EB0D
:10815000025585EACE710AD05FEA440C18BF24F0BC
:10816000004450F1000041F1000120EAD47040F2D7
:10817000FE7C624500D270BDA84214BF4FF080441F
:108180004FF04044002E08BF0024BEF1806FA8BF0E
:10819000A1F1C041BDE8704080F282804FF0000044
:1081A00001F1C04101F0004170479EEA0C0F0CEA5A
:1081B000131518BF95EA0C0F06D04FF0000081EAA6
:1081C000030E0EF0004170BD00F01CF88900013E66
:1081D00000F007B800F009B84FEA430C5FEA5C5CB6
:1081E00008D081EA030100F05BB84FEA410C5FEA76
:1081F0005C5CF6D14FF00000014970470000FF07BA
:108200000000F87F0EF1020E2EF0030E5EF8046BF4
:10821000364205D4012A43EB030515F5001F12D899
:10822000012841EB010C1CF5001F0CD80ED14FEAC0
:10823000D17C15F5001F0CEB4C0C0CF1020C08BFA7
:108240004CEBD37C04E04FF0080C01E04FEAD37C08
:108250000CEB4C0526FA05F606F00706B6F1040C01
:1082600006D20EEB860CBDE870404CF0010C604766
:10827000DFE80CF0090B02024FF000414FF0000064
:10828000A1F5002170BD19461046012851EB0104EB
:1082900018BFD4F5001484BF002001F0004170BD68
:1082A0000808A0F500114FEA3101704743004FEA7A
:1082B000D30C4FEA3C0C43401FBF40070CF1605108
:1082C00013F0FE4F70471CF0006F03D100200CF03C
:1082D000004170470CF0004343EA507010B540EA8B
:1082E000CC0000F096FA00BF000000924FEA0001B7
:1082F000FFF7D6BF4FF000414FF00000A1F500217D
:108300007047000090EA010F48BF81F0004100F182
:108310000483421A3CBF801A89184FEAD0524FF0AA
:108320007F4C1CEA410FA2EBD15318BF9CEA026FAD
:1083300000F03B804FF0004C4CEA00204CEA012159
:1083400021FA03FC10EB0C0C1ED202F1FF325FEAA3
:108350001C2040EBC25038BF70471CF07F0F4FEA23
:10836000400C18BFBCF17F4F38BF7047C3F12003EA
:10837000994008BF20F00100BCF17F4F38BF704723
:10838000A0F1C04000F08BBA4FEA3C00000A40EB7D
:10839000C25028BF1CF0FF0F4FEA400CE6D018BFB8
:1083A000BCF17F4F38BF7047EAE79CEA026F05D007
:1083B00010EA5C0F08BF00F00040704710B500F0F5
:1083C00028FA00BF64FBBE3E014800F016BB00BFA8
:1083D0000000C07F401058BFC0F14040491058BF56
:1083E000C1F140418142EFF3008070474FF47F0CB0
:1083F0001CEAD0121EBF1CEAD11392EA0C0F93EABA
:108400000C0F00F0858090EA010F48BF42F48072A3
:1084100040F4000C41F400002CF07F4120F07F403C
:1084200000B58142A2EB03020FF2081CACEB504EE8
:10843000C0F100009EF800E04FEA4E0E00FB0EFC7B
:1084400038BF49004FEA2C1C02F5FA020CFB0EF370
:108450004FEACE1E4FEA112C4FEAC1210EEB635EAC
:1084600042EB22420EFB0CFC4FEA1C5300FB0311B3
:108470004FEA112C4FEA01310EFB0CFC4FEADC4CA9
:1084800000FB0C11C14228BF09184CEB03335DF807
:1084900004EB10EB410143EBC250B2F57C0F38BF47
:1084A000704729D512F0F00F1CBF00F1C04000F05A
:1084B00000407047008182838485868788898B8C01
:1084C0008D8E8F919293959697999A9C9D9FA0A23D
:1084D000A3A5A7A8AAACAEB0B2B3B5B7B9BCBEC08D
:1084E000C2C5C7C9CCCED1D4D7D9DCDFE2E6E9EC2E
:1084F000F0F3F7FAFE0000004FEA400C0CF1807C2C
:10850000BCF17E4F28BF7047B0F1C04000F0C7B942
:1085100090EA010F0CEAD11348BF42F48072624521
:1085200038BF634507D213F47F0F16D080EA0100ED
:1085300000F00040704710B500F06BF9097EFC3E7A
:1085400000F005B880EA010000F00040704780EAC2
:10855000010000F0004000F0A2B912F47F0F04BF48
:108560000248704780EA010000F099B90000C07F1E
:1085700050EA010C00F113801CF5000F58BFBCF548
:10858000000F01D48842704707D710F5000F58BF7D
:1085900011F5000F15D488427047894270471CF5C9
:1085A000000F04D5BCF5000FF7D5814270474FF09E
:1085B000807C1CEB400F38BF1CEB410F01D2814285
:1085C000704710B500F025F9922449004FF0005093
:1085D0004FF08051FFF7FEBE41000B0ED3F19E021B
:1085E00008D950F400034FEA032323FA02F048BFEE
:1085F0004042704710B500F00CF900BF499224804A
:10860000002070476FF0004282EA200070470000AF
:10861000C10DD1F19E0206DB4FEA002343F0004377
:1086200023FA02F07047004207D54FEA4001B1F14A
:10863000FE4F02D24FF00000704710B500F0E9F88D
:1086400049922480002070476FEA200070470000A4
:1086500010F0004148BF4042B0FA80F310FA03F234
:10866000C3F19D030BD051EAC35101EB1220530615
:1086700038BF704700F1010008BF20F001007047CB
:10868000B0FA80F310FA03F2C3F19D030AD0D905C2
:1086900001EB1220530638BF704700F1010008BFFC
:1086A00020F001007047000050EA010C00F1138037
:1086B0001CF5000F58BFBCF5000F01D4884270476D
:1086C00007D710F5000F58BF11F5000F15D48842D9
:1086D0007047894270471CF5000F04D5BCF5000FA8
:1086E000F7D5814270474FF0807C1CEB400F38BFBC
:1086F0001CEB410F01D28142704710B500F089F8A0
:10870000922449004FF000504FF08051FFF762BEB5
:108710004FF47F0C1CEAD0121EBF1CEAD11392EA60
:108720000C0F93EA0C0F00F0478090EA010F48BF4E
:1087300042F480724FF0004C4CEA00204CEA0121D8
:1087400002EB0302A0FB0113A2F50002002918BFEF
:1087500043F001035B0028BF4FEA330342EB2242A0
:108760005FEA132C4CEBC2502EBFBCEB436FB2F54B
:108770007C0F70474FEA036CBCF1004F08BF20F03C
:108780000100B2F57C0F38BF70470BD582F0FF02B5
:1087900012F5803FC8BF704700F1C040D8BF00F05D
:1087A0000040704700F5000C5FEA4C0C48BF704772
:1087B000B0F1C04000F073B890EA010F0CEAD11399
:1087C00048BF42F48072624538BF634504D280EAF4
:1087D000010000F00040704710B500F01AF800BF2B
:1087E0008900013E00F007B800F009B85FEA410CCB
:1087F0005FEA1C6C08D080EA010000F050B85FEA24
:10880000400C5FEA1C6CF6D14FF00040A0F58000F0
:1088100070470EF1020E2EF0030E5EF8044B244258
:1088200004D44FEA4102B2F17F4F11D84FEA40031E
:10883000B3F17F4F0CD80ED14FEAD07CB2F17F4F0D
:108840000CEB4C0C0CF1020C08BF4CEBD17C04E09F
:108850004FF0080C01E04FEAD17C0CEB4C0324FAFA
:1088600003F404F00704B4F1040C06D20EEB840CFC
:10887000BDE810404CF0010C6047DFE80CF0070841
:1088800002024FF00040A0F5800010BD08464200F3
:1088900018BFD2F1807288BF00F0004010BDFF21E8
:1088A00041EAD050C005704751EA000C00F1138036
:1088B0001CF5000F58BFBCF5000F01D48142704772
:1088C00007D711F5000F58BF10F5000F15D48142DE
:1088D0007047894270471CF5000F04D5BCF5000FA6
:1088E000F7D5884270474FF0807C1CEB410F38BFB2
:1088F0001CEB400F01D28842704780EA010081EAF8
:10890000000180EA0100FFF7F8BE000090EA010FC5
:1089100048BF81F000413FF5FCAC421A04D882F018
:108920000042A0EB020011444FEAD0524FF07F4CBE
:108930001CEA410FA2EBD15318BF9CEA026F4AD048
:108940004FF0004C4CEA00204CEA012121FA03FCD4
:10895000B0EB0C0C0FD412F0FE0F36D05FEA4C00D7
:108960001DD5001240EBC25038BF70471CF03F0FBE
:1089700018BF70470BE0A2F101025FEA1C2040EB38
:10898000C25038BF70471CF07F0F18BF7047C3F14B
:108990002003994014BF401E20F00100704780085A
:1089A0004FEA122308BF7047B0FA80FCA2EB0C021A
:1089B000CCF1280C60FA0CF093EA122F04BF00EB04
:1089C000C25070474FEAC3707047130A5FEADC1069
:1089D00008BF7047F6E79CEA026F04D010EA5C0F0C
:1089E00008BF0020704710B5FFF713FF40DFF63EC9
:1089F00081F000407047F7F780BE0CF00F03092BA1
:108A000008BF082000F051800A2B0BD0082B18BF9C
:108A1000704708BF1CF0400F0AD04FF000004FF025
:108A2000000170471CF0400F18BF4FF00040704726
:108A30001CF0100F08D020F0704300F07F4242EA93
:108A4000D3014FEA4370704700F0604021F07F424D
:108A500042EA000201F07F4040EA727070474FF036
:108A6000FF0212EAD0521CBF92F0FF038B42C2BF3A
:108A7000D14200EBC1507047002A0AD0002B0BD026
:108A8000002900F00040A4BF40F0FE4040F4000088
:108A9000704700F00040704743024FF00B0C18BFC6
:108AA0004CF0806C7FF490AC70471CF4801F11D0A8
:108AB0001CF4E02F03D06FEACC31490070474FF02F
:108AC0004050EFF3008222F0704242EA000282F34B
:108AD000008870474FF00000704701020203040550
:108AE000060708090A0B0C0D0E0F101000000000FD
:108AF000000000000102030406070809000000004E
:108B0000010203040000000000000000002F00002C
:108B100000000700070000147F147F1400242A7F40
:108B20002A120062640813230036495522500000BF
:108B30000503000000001C224100000041221C002F
:108B40000014083E08140008083E0808000000A0B1
:108B500060000008080808080000606000000020AD
:108B600010080402003E5149453E0000427F40008B
:108B7000004261514946002141454B310018141211
:108B80007F10002745454539003C4A4949300001DE
:108B90007109050300364949493600064949291E2D
:108BA000000036360000000056360000000814228F
:108BB000410000141414141400004122140800028F
:108BC0000151090600324959513E007C1211127CB4
:108BD000007F49494936003E41414122007F4141E1
:108BE000221C007F49494941007F09090901003ED3
:108BF0004149497A007F0808087F0000417F410011
:108C0000002040413F01007F08142241007F404086
:108C10004040007F020C027F007F0408107F003E6E
:108C20004141413E007F09090906003E4151215E54
:108C3000007F091929460046494949310001017F51
:108C40000101003F4040403F001F2040201F003FE7
:108C50004038403F00631408146300070870080799
:108C600000615149454300007F41410000552A55AC
:108C70002A55000041417F00000402010204004027
:108C80004040404000000102040000205454547849
:108C9000007F484444380038444444200038444469
:108CA000487F00385454541800087E090102001807
:108CB000A4A4A47C007F080404780000447D400044
:108CC000004080847D00007F102844000000417F28
:108CD0004000007C04180478007C08040478003804
:108CE0004444443800FC242424180018242418FC8C
:108CF000007C0804040800485454542000043F44F5
:108D00004020003C4040207C001C2040201C003CB7
:108D10004030403C004428102844001CA0A0A07C07
:108D2000004464544C44141414141414000000003F
:108D3000000000000000000000000000000000F83B
:108D400000000000000000333000000000100C069E
:108D5000100C0600000000000000000040C0784039
:108D6000C0784000043F04043F040400007088FC05
:108D700008300000001820FF211E0000F008F0005D
:108D8000E018000000211C031E211E0000F00888CE
:108D9000700000001E2123241927211010160E0038
:108DA000000000000000000000000000000000E0E3
:108DB00018040200000000071820400000020418F8
:108DC000E00000000040201807000000404080F054
:108DD000804040000202010F01020200000000F08A
:108DE000000000000101011F01010100000000005E
:108DF0000000000080B070000000000000000000D3
:108E0000000000000001010101010101000000005B
:108E100000000000003030000000000000000000F2
:108E200080601804006018060100000000E01008CF
:108E30000810E000000F102020100F00001010F8A4
:108E4000000000000020203F2020000000700808E3
:108E50000888700000302824222130000030088863
:108E6000884830000018202020110E000000C0208B
:108E700010F8000000070424243F240000F80888AC
:108E8000880808000019212020110E0000E0108839
:108E900088180000000F112020110E00003808086B
:108EA000C83808000000003F00000000007088087B
:108EB00008887000001C222121221C0000E01008FC
:108EC0000810E0000000312222110F00000000C055
:108ED000C0000000000000303000000000000080F2
:108EE00000000000000080600000000000008040E2
:108EF00020100800000102040810200040404040FB
:108F0000404040000404040404040400000810204D
:108F10004080000000201008040201000070480892
:108F20000808F0000000003036010000C030C828FA
:108F3000E810E0000718272423140B000000C038B5
:108F4000E0000000203C23020227382008F888882F
:108F500088700000203F202020110E00C03008083B
:108F600008083800071820202010080008F8080812
:108F70000810E000203F202020100F0008F888880B
:108F8000E8081000203F20202320180008F88888D7
:108F9000E8081000203F200003000000C03008084F
:108FA0000838000007182020221E020008F80800D8
:108FB0000008F808203F210101213F20000808F89F
:108FC000080800000020203F2020000000000808C2
:108FD000F8080800C08080807F00000008F888C082
:108FE00028180800203F20012638200008F8080033
:108FF00000000000203F20202020300008F8F8006A
:10900000F8F80800203F003F003F200008F830C07B
:109010000008F808203F200007183F00E01008086B
:109020000810E0000F10202020100F0008F808089A
:109030000808F000203F210101010000E0100808AD
:109040000810E0000F18242438504F0008F88888D2
:1090500088887000203F2000030C302000708808B2
:10906000080838000038202121221C00180808F8C0
:10907000080818000000203F2000000008F8080041
:109080000008F808001F202020201F000878880012
:1090900000C83808000007380E010000F80800F882
:1090A0000008F800033C0700073C0300081868802C
:1090B0008068180820302C03032C30200838C800A2
:1090C000C83808000000203F2000000010080808F1
:1090D000C83808002038262120201800000000FE93
:1090E000020202000000007F40404000000C30C03F
:1090F00000000000000000010638C000000202026B
:10910000FE000000004040407F000000000004021C
:109110000202040000000000000000000000000047
:109120000000000080808080808080800002020437
:10913000000000000000000000000000000080802F
:10914000808000000019242222223F2008F800809D
:1091500080000000003F112020110E000000008060
:1091600080800000000E11202020110000000080EF
:109170008088F800000E112020103F200000808021
:1091800080800000001F222222221300008080F035
:10919000888888180020203F202000000000808060
:1091A00080808000006B94949493600008F80080A5
:1091B00080800000203F210000203F200080989800
:1091C000000000000020203F202000000000008060
:1091D0009898000000C08080807F000008F80000A0
:1091E00080808000203F24022D302000000808F8F5
:1091F000000000000020203F2020000080808080B0
:1092000080808000203F20003F20003F8080008041
:1092100080800000203F210000203F20000080804F
:1092200080800000001F202020201F008080008000
:109230008000000080FFA12020110E0000000080AF
:1092400080808000000E112020A0FF8080808000A0
:109250008080800020203F212000010000008080CD
:10926000808080000033242424241900008080E0C2
:10927000808000000000001F20200000808000008F
:1092800000808000001F202020103F208080800070
:109290000080808000010E30080601008080008080
:1092A000008080800F300C030C300F0000808000A5
:1092B000808080000020312E0E31200080808000D0
:1092C0000080808080818E70180601000080808080
:1092D000808080000021302C22213000000000001E
:1092E000807C020200000000003F404000000000BF
:1092F000FF00000000000000FF0000000002027CF0
:10930000800000000040403F000000000006010116
:10931000020204040000000000000000040444C431
:109320004F4444C424242FB424040400404424247F
:10933000150C04FE040C1524244440000000F849D8
:109340004A4C48F8484C4A49F800000010101312E3
:10935000121212FF1212121213101000002020A875
:109360006C2A3928A82A6CA820200000028281904B
:10937000924A4945242210080102020090523410FA
:10938000FF10345280708F0808F80800829A5663E4
:1093900022528E008040330C3340800000007E005B
:1093A00000FF0040300F04146404000040407E427F
:1093B000427E4242427E42427E4040001060028C29
:1093C00000FE02F202FE00F800FF000004047E012D
:1093D0008047300F10270047807F00000000F8888A
:1093E000888888FF88888888F800000000001F08A7
:1093F0000808087F888888889F80F0001010D0FFB8
:10940000901000FE020202FE00000000040300FFB4
:109410000083601F0000003F40407800101010FFE4
:109420009020984828090E2848A818000242817FF9
:109430000040404242427E424242400040504E483C
:1094400048FF48484840F80000FF000000003E0286
:1094500002FF12221E000F40807F000084E45CC4E3
:109460000008C8398E0808CC3B880800003F103F30
:1094700000635A46E100635A46E10000809090483C
:109480004C5724E424544C44808080000042221233
:109490000A42827F02020A122242000000000414E3
:1094A00064040CB402024233020000004041211166
:1094B000090503FF03050911214140001010D0FFE9
:1094C000900010919690F09094931000040300FF88
:1094D000000104040404FF040404040000FE02224A
:1094E000DA0600FE22222222FE00000000FF081001
:1094F0000847407F424242427F404000000000FE59
:1095000042424242C24242427E0000008040300F4E
:1095100000000000030C1020408080001060028CCE
:109520000000FE9292929292FE00000004047E01DE
:10953000407E42427E427E42427E40000000FC2449
:109540002424FC252624FC242424040040308F807D
:10955000844C55252525554C8080800000FE225ADC
:109560008600FE9292929292FE00000000FF040894
:109570000700FF4020030C1422414000008060F8E7
:109580000710901011161010D0100000010000FFFD
:109590004040415E4040704E414040004262524A6D
:1095A000C6425262C200F80000FF000040C44444BA
:1095B0007F24242420000F40807F0000404042CCC4
:1095C00000101010907F9010101010000040201F0D
:1095D0002048444241404041424C4000404042CC3F
:1095E00000202222A2622222222000000040201F0E
:1095F00020444E4544444445464C4000001088C435
:10960000330040424242C24242424000020100FF57
:109610000000000040807F00000000001010D0FF1C
:109620009014E4AFA4A4A4AFE4040000040300FF7A
:1096300000894B2A1A0E1A2A4B888000101090902D
:109640009090901010FF1010111610000020602054
:109650003F10101000030C102040F8000000C04024
:1096600040407F48484848C8080800008040370408
:10967000041464041464040710E000004044C4446B
:109680004444401010FF101010F00000103C131064
:1096900014B840300E014080403F00001088C433B1
:1096A00000FE12D252527F5151D110000100FF40F2
:1096B000300F00FF4A4A4A4A4AFF0000048484FCF3
:1096C000848400040484E41C840404002060201FBB
:1096D000101004020100FF00000106004040407C21
:1096E000404040FF44444444444040008090884609
:1096F0004040202F1010080402000000808080806D
:10970000FF8080A09088848280808000000000001C
:10971000FF402112040810202040400008080808DB
:1097200008F8898E8888888808080800008040200A
:10973000180700004080403F0000000000F80808C3
:109740000CCA494848C8080808F8000000FF000093
:10975000001F0808081F0040807F0000000202C2AE
:10976000020202FE82828282820200004040407F2A
:109770004040407F40404040404040000000FC24CA
:1097800024E42424222222A36200000040308F809F
:109790004040231408142241408080000484E45C8B
:1097A00044C42010E82724E4342CE00002017F1098
:1097B000103F80601F09093F49897F00404042CC2B
:1097C0000000000000FF0000000000000000003F5B
:1097D0009048201807000718204080000202FE92DF
:1097E0009292FE0206FC040404FC000008180F0814
:1097F0000804FF0484402718274080001060020CF2
:10980000C000E22C203F2028E600000004047C0376
:109810000000FF09090949897F000000001088C481
:10982000330040424242C24242424000020100FF35
:109830000000000040807F00000000000000F010E9
:10984000101010FF10101010F000000000000F04A6
:10985000040404FF040404040F0000000000E2827A
:1098600082828282828282FE0000000000003F40ED
:10987000404040404040404040780000100C0424EC
:10988000242425262424242404140C00008181414E
:10989000310F0101017F818181F100000000F88812
:1098A0008888880808FF08090AC8080080601F0027
:1098B00010201F80402116182641F800404042CC5D
:1098C0000040A09E8282829EA02020000000003FD7
:1098D000908840432C10284641808000001715D501
:1098E0005557557D555755D5151700004040407FB9
:1098F000555555555555557F4040400000F80106D7
:1099000000F0121212F2020202FE000000FF00003C
:10991000001F1111111F0040807F000000FE225A1D
:109920008600027A4A4A4A4A4A7A020000FF04083C
:109930000700FF090B0D790D4B897F001060028C29
:10994000000E22120AC20A12220E000004047E0136
:109950002021110905FF050911212000201008F719
:1099600054545454545454F40404000080909049C6
:109970004D57252525554D45808080001010D0FF7E
:109980009010804828090E0828488800040300FF2A
:1099900000018080432C102C4380800000020CE0EA
:1099A0004020F84F4849FE484848080004047F001A
:1099B0000000FF2222223F222222200000404244B7
:1099C0005840407F40405048C6000000004044449A
:1099D0004444444444444444FF0000000808E82947
:1099E0002E28E80808C80C0BE80808000000FF094A
:1099F00049897F00000F40807F00000040484848B0
:109A0000FF484800C4444444FC00000080601F201C
:109A10007F4444404F505050505C40000240000092
:109A2000000000A00000000005400000000000C889
:109A3000000000000C4000000000409C00000000FE
:109A4000194000000020BCBE0000000034400000AF
:109A5000BFC91B8E00000004B5400000504BCFD0A2
:109A60006607E2CF010000006C4100003E8251AA6F
:109A7000DFEEA73401000000D9420000DCB5A0E20F
:109A80003A301F97FFFFFFFFB4450000FD25A0C837
:109A9000E9A3C14FFFFFFFFFFF3F00000000008070
:109AA00000000000FF3F00000000008000000000F8
:109AB000EC9A000800000020D00100006C010008B2
:109AC000349B0008D001002050140000C801000899
:109AD0001C00000043000000F8FFFFFF0C00000026
:109AE0000E0000000F0000002E00000001543201A3
:109AF0008210D324F4C2641B05012C0B1A32FF48D8
:109B0000C123204E23409C23A00F8BB80B080930A3
:109B10009E0938D8091A3E692023D8046A02B42263
:109B2000031AB0100922866914091FA21319A10291
:049B300017B1000069
:0400000508000131BD
:00000001FF
